:10000000F01F001055380000513800005138000032
:100010005138000051380000513800000000000045
:100020000000000000000000000000005138000047
:100030005138000000000000513800005516000043
:1000400025140000251400002514000025140000CC
:1000500025140000251400002514000025140000BC
:1000600025140000251400002514000025140000AC
:10007000251400004D3800004D3800004D380000B8
:100080000D170000251700003D1700005517000050
:100090004D3800001D1800004D3800004D3800009C
:1000A0004D3800004D3800004D3800004D3800003C
:1000B0004D3800004D3800004D3800004D3800002C
:1000C00008B500230B60036000F01AFE08BD08B5F8
:1000D0000A20002101F0BAFA08BD000038B5094B2A
:1000E0000D1C041C1968012001F060FB012001F0C7
:1000F0003DFB291C201C02F02BFF012001F046FBD8
:1001000038BDC046BC04001070B5054E051C0E2459
:10011000013C295D301C01F09DFD002CF8D170BD23
:10012000843A000038B5164801F094FD154C201CA7
:10013000FFF7EAFF144D4221281C01F08BFD201C23
:100140000E30FFF7E1FF4321281C01F083FD201C46
:100150001C30FFF7D9FF0D4801F07CFD201C2A3030
:10016000FFF7D2FF281C4E2101F074FD201C38300F
:10017000FFF7CAFF616D064801F06CFD38BDC0464F
:10018000873A0000C40400108D3A0000943A000041
:100190009A3A000010B5084B041C1968012001F0C0
:1001A00005FB012001F0E2FA201C02F061FE0120B3
:1001B00001F0ECFA10BDC046BC04001008B50020E8
:1001C000FFF7E8FF08BD000010B5041C00F024FC98
:1001D000201C00210322034B00F012FD00F026FC3E
:1001E00010BDC0460000001008B5021C02490348BB
:1001F00001F030FD08BDC046AE3A0000A63A00004E
:1002000013B59620000201F047FB1248FFF7DCFF10
:10021000FFF7D4FF1048FFF7E7FF002401F0DAFBF7
:10022000002803D001F018F8002409E00A2001F0AA
:100230003DFA684601A9FFF743FF009B002B03D15D
:10024000064B01349C42E9DDFFF7B8FF044801F09A
:1002500001FD13BDB73A0000C63A00006F17000059
:10026000CC3A00007047000000B5074B89B01A78FF
:10027000064B68461B78064901F0F7FC6846FFF715
:10028000A3FF09B000BDC046C8010010080000105F
:10029000D73A000013B5FFF7E7FFFFF78FFF002401
:1002A000684601A9FFF70CFF009B002B2CD0182BF0
:1002B00021D004DC142B0DD0152B20D104E0342BDD
:1002C00012D0352B1BD107E0134B00241A783E2A9D
:1002D00016D806E0104B08E0104B00241A78062AC6
:1002E0000ED801321A700BE00C4B1C78002C07D092
:1002F000013C1C7003E0FFF761FF282400E00024AC
:1003000000F076FBFFF7B0FFC820013401F0CEF912
:100310001D2CC5DD13BDC046C8010010080000102B
:1003200073B5124B041C1249186803F015FB1149F0
:100330000090114A114B201C01F097FC00F0C2FD07
:10034000002812D000F0DAFDFA218900051C03F024
:1003500003FB061C201C01F0D5FC094B201873433D
:100360000849EB18321C01F080FC73BDC00400107A
:1003700040420F00E53A0000AE3A0000F23A0000B9
:1003800018FCFFFFF63A000070B5051C0C1C161C8B
:1003900000F042FB291C201C0022064B00F030FC20
:1003A000301C01210922044B00F02AFC00F03EFB26
:1003B00070BDC046000000100C00001038B50D1CC8
:1003C000041C00F0F4FA2A1C0120211CFFF7DCFFBA
:1003D000034B00225A60034A943212689A6038BD77
:1003E000600C0010C404001010B590B0041C6846E6
:1003F000FFF796FF69466A46201CFFF7C5FF10B05D
:1004000010BD000073B518200021FFF767FE464EAF
:10041000464D00249836012001F0B8F9002C01D097
:10042000002000E00620012101F010F9684601A932
:10043000FFF746FE009B002B21D1002CF0D1336842
:10044000002B0DD03A4B00941A6811321A6004E068
:1004500002F0B8FC009B01330093009B102BF7DDEA
:10046000344BED18DED518200021FFF737FE2E4B58
:1004700094331C6863425C4100F082FACEE7002CA2
:1004800006D0182BC7D12C48FFF7AEFE00F0D6FAE5
:10049000009B182B2BD1019B00220192822B22D092
:1004A00004DC322B0ED0732B20D119E0832B0FD01C
:1004B000C22B1BD1214B196801311960022916D1B9
:1004C0001A6014E01E4B01201B68C01A00F03CFDAE
:1004D0000120FFF789FFFFF771FEFFF7F8FD06E047
:1004E000FFF78EFE03E0FFF7D5FE00E0019300F07A
:1004F00017FD144B0120196801F058F9012001F093
:1005000035F90098019902F023FD074B94331B68DD
:10051000002B03D100F034FA012402E003F034F997
:100520000024024D77E7C046C404001020BF02003B
:10053000F80200100CFEFFFF013B0000A0010010BC
:1005400018000010BC04001013B501F00BFC00F003
:10055000A3FB00F073FA00200421012200F0A4FEA6
:100560000020021C042100F0EDFE002005210122E4
:1005700000F09AFE0020021C052100F0E3FE134863
:10058000002100F003FF0021114800F0FFFE00F001
:1005900029FC00F06DFE3C24201CFFF725FF013CE8
:1005A0001E2001F083F8022CF6D101F023FC02F0AA
:1005B00027FB1E2300930F23019306480649074A91
:1005C000074B02F0D7FBFFF71DFFC04698400440E1
:1005D0009C40044009380000C1000000BD03000039
:1005E000F802001000B500E001300378202BFBD0AA
:1005F00000BD00B5031C303BDAB2092A01D8181C33
:1006000008E020231843031C613B5738052B01D910
:100610000120404200BD70B50E1CFFF7E3FF00252E
:10062000041C06E0FFF7E5FF002805DB2D0105436C
:10063000013420780028F5D13560201C70BD000001
:1006400008B500F05BFC011C014801F003FB08BD8C
:100650000B3B000000B5C300181A064BC018072357
:10066000013BC25C002A03D1002BF9D1012000E03C
:10067000002000BD600500107FB5194801F0EAFABE
:1006800000250326354219D1281CFFF7E3FF002877
:1006900010D0681CFFF7DEFF00280BD0A81CFFF766
:1006A000D9FF002806D0E81CFFF7D4FF002801D0AE
:1006B00004350FE00B48291C01F0CCFA291C6846D0
:1006C00001F0BCFB6846FFF71FFD074801F0C2FAC6
:1006D0006C1C251CFF2DD5DDFFF724FD7FBDC0461A
:1006E000AE3A0000173B0000E77D000070B50E1C1D
:1006F000FFF778FF0D25041C2078FFF77AFF00280C
:1007000007DB01347055013DF6D2201CFFF76AFF6C
:1007100000E0002070BD000030B5464C87B0236873
:100720000868002B06D1444801F094FA02F068FAF8
:10073000012357E0012B12D1037A202B07D0002B85
:1007400005D03E49082201F0F0FA002803D1394BC8
:100750001A6801326AE03A4801F07CFA5EE00378F8
:10076000412B1BD1374C0230211CFFF7BFFF002863
:1007700054D00378422B51D1211C02300E31FFF7A7
:10078000B5FF00284AD00378432B47D1211C023003
:100790001C31FFF7ABFF002849D13FE04D2B23D19F
:1007A000294D0230291CFFF7A1FF002836D003781D
:1007B0004E2B33D1291C02300E31FFF797FF002852
:1007C0002CD00378472B29D1023005A9FFF723FF4E
:1007D000059B002B22DB2A3D6B651C481C4901F060
:1007E00039FA0023236022E005A9FFF714FF0378FC
:1007F000041C202B01D0002B10D10025201C01A9A6
:10080000FFF774FF0599041C691801A801F02AFB81
:10081000002C03D00135042DF0D108E002F0F0F9EE
:100820000A480C4901F016FA024B00221A6007B080
:1008300030BDC046D0020010203B0000AE3A0000A0
:10084000363B0000C4040010EE040010423B0000E0
:100850004C3B00004F3B000037B54C6824E0201CA7
:10086000FFF7C0FE01A9FFF7D6FE019B041C002B79
:100870001DD0D8B2FF2B09DD00F0DEF9051C019870
:100880000012C0B200F0D8F9019003E000F0D4F9F2
:10089000002501900198002802D0291CFFF71EFCBA
:1008A00023785A1E9341E4182378002BD7D137BD03
:1008B00008B5064A012113784B40137001D0044952
:1008C00000E00449044801F0C5F908BDB103001077
:1008D000083B0000563B00005A3B000070B5051C69
:1008E00001200821021C00F02DFD07240126012013
:1008F0000821002200F026FD2A1C2241324000205F
:10090000022100F01FFD01200821021C00F01AFD49
:10091000013CECD270BD10B50021041C0A1C022061
:1009200000F010FD201CFFF7D9FF10BDF7B5012323
:1009300000930023019372B66C46061C02AF01CCF3
:1009400050235B421843C0B2FFF7E5FF0020FFF7DA
:10095000E2FF1020FFF7DFFFE020FFF7DCFF0025BC
:1009600002200021012200F0EDFC705D0135FFF74F
:10097000B5FF842DF4D18436BC42E0D162B6F7BD18
:1009800008B5AC20FFF7C7FFAE20FFF7C4FFA520D6
:10099000FFF7C1FF08BD38B50D1C041C012200F093
:1009A00083FC291C201C012200F0CCFC38BD08B5BA
:1009B000AF20FFF7B0FFA420FFF7ADFF08BD08B5DB
:1009C000AE20FFF7A8FF08BD10B5041CF820FFF704
:1009D000A2FF201CFFF79FFF10BD10B5041C812053
:1009E000FFF799FF3F202040FFF795FF10BD000063
:1009F00008B5074B20201B781843FFF78CFF0A200F
:100A000000F054FE034B1878FFF7E7FF08BDC0461F
:100A100008000010C801001008B584220248002117
:100A2000520001F04FF908BDB203001008B50248AA
:100A3000FFF77CFF08BDC046B203001008B50120D7
:100A40000821FFF7A8FF00200221FFF7A4FF0220E2
:100A50000021FFF7A0FF02200621FFF79CFF0320E3
:100A6000011CFFF798FF0320011C002200F06AFC24
:100A700002200621002200F065FC0621012202204E
:100A800000F060FCFFF7C8FFFFF7D0FFA220FFF7E0
:100A900042FFA020FFF73FFFC020FFF73CFF0020F0
:100AA000FFF792FF0A2000F001FE4020FFF733FF1E
:100AB0002C20FFF730FF322000F0F8FD2E20FFF74A
:100AC0002AFF322000F0F2FD2F20FFF724FF0A203A
:100AD00000F0ECFDFFF78CFFAF20FFF71CFFA42018
:100AE000FFF719FF08BD000000B50F290ED88328B5
:100AF0000CD8CB08842253430722C0181140044B62
:100B000080220A41111C1A5C1143195400BDC046D1
:100B1000B2030010F0B55B18DBB216E08425CC08F8
:100B20006C4307270F40802504193D41EFB2A618FA
:100B30009C4605E0064BE5182B7801343B432B70AF
:100B4000B442F7DB01316346C9B29942E6D3F0BD46
:100B5000B2030010F0B589B0059106921C1C5D68C7
:100B6000DB78834202D22478039444E0A378234ABA
:100B7000C01A0023954209D14300181803234519D0
:100B8000039309E02A7801330232AD188342F9DB7E
:100B900069782B7803910235EB18002604930196AF
:100BA00025E0082F05D1049A954224D02E780027FD
:100BB0000135F30706D5029A069B0798D118C9B2EA
:100BC000FFF792FF0299761001310291013707E099
:100BD000002202920199059A08278B18DBB207932D
:100BE000637802999942DCDB019A01320192019B00
:100BF00003998B42ECDB039809B0F0BD693B000020
:100C0000F0B585B0061C0C1C0292039301F07AF833
:100C100000250190832708E0705D211C029A039B48
:100C2000FFF798FF013024180135A74202D3019B3A
:100C30009D42F1D305B0F0BD00B50F230209184065
:100C40008000031F00D52833002B0EDB511E03202C
:100C5000884280414042002807D1242B06DC042131
:100C60008A1A0349CB18985C00E0002000BDC046FA
:100C70003240000070B5064E051C0024A05D054BF7
:100C8000291CC018013400F081FB0A2CF6D170BD7C
:100C90006E40000000400440F8B51020FFF7EAFF66
:100CA000094C271C143725786678281C311C002233
:100CB00000F0FAFA0234281C311C012200F042FB39
:100CC000BC42F0D1F8BDC0465A400000F8B50B4C0C
:100CD000271C143725786678281C311C012200F067
:100CE000E3FA0234281C311C002200F02BFBBC422A
:100CF000F0D10020FFF7BEFFF8BDC0465A4000000B
:100D0000F0B589B0002404900591FFF7C5FF0220DB
:100D1000072101220694079400F0C6FA0220072159
:100D2000221C00F00FFB201C0B2100F0E1FAA04276
:100D300002D11823069301240021264D03916A78DD
:100D40002F78111C0192381C012200F0ADFA381CDA
:100D50000199002200F0F6FA03231F4E029314E0DB
:100D60003078717800F0C4FA002807D103991B4A43
:100D7000A3008A5C183369465A500134029A039BD7
:100D8000013A013302920393023EE30F0021012254
:100D9000A2424B41DBB28B4202D0029B8B42DFDA94
:100DA000381C0199002200F07FFA0199381C0122B9
:100DB00000F0C8FA0A4902358D42C0D1201E06D083
:100DC000069B049A05991360079B01200B6009B0EC
:100DD000F0BDC0465A4000003040000032400000E4
:100DE0006E40000008B50120021C0B2100F05CFAE7
:100DF00001200B21002200F0A5FA0320022101228C
:100E000000F052FA03200221002200F09BFA08BDF4
:100E100037B5234B10211A68051C8A431A60214BF1
:100E20008022196892010A431A6001200B210022D6
:100E300000F03AFA01200B21002200F083FA1A4B4D
:100E40009F211A68194C8A431A601A6818491A6057
:100E5000184B186802F080FD8023000218432A1CFA
:100E600020600221032000F06DFA142000F01EFC27
:100E70002368FF229343236023680F4A13432360B0
:100E80000E4B1A680192019A002AFADA22680C4B7A
:100E900013402360FFF7A6FF01980004800D3EBDBC
:100EA00038820440808004409840044000C00140E3
:100EB00000093D00C0040010800000012CC001406A
:100EC000FFFFFFF810B50C4C2068002813DA002053
:100ED0002060FFF79DFF0A280ADC0120FFF798FF3A
:100EE0000138C023FF385B00984201D801232360FA
:100EF000FFF778FF206810BD1400001008B5FFF759
:100F0000E1FF011E08D00120FFF782FF011E03D080
:100F1000024802F021FD011C081C08BD50BB120054
:100F200008B5FFF7CFFF00280AD0FFF7E7FFFA2246
:100F3000031C0021C00FD2009A424841014B1860A7
:100F400008BDC046CC01001010B500280DD0254BBF
:100F500080211A688A431A60234A012311681942C2
:100F6000FCD0224B03221A6001E0204B1860204B7A
:100F7000012200211A6019601A6019681142FCD020
:100F80001C4B01221A601C4A80211468490221432B
:100F900011601A1C002804D1124B802419682143C7
:100FA0001960164B196888421AD01860002801D0C1
:100FB000134800E01348116802F080FC124C212114
:100FC000206002F0C9FC114B18609620000200F06E
:100FD00063FCFA212068890002F0BEFC00F04CFBA3
:100FE00010BDC046388204400C800440708004402C
:100FF0007480044078800440808004401800001011
:10100000006CDC02001BB700C0040010BC04001020
:1010100008B500F03BF9134B00211A68120B1203BC
:101020001A60114B1A68120B12031A600F4B1A68E0
:10103000120B12031A600E4B1A68120B12031A607D
:101040000C4B012219600C4B1A6019601A60196868
:101050001142FCD0094B23221A600120FFF774FFD4
:1010600008BDC04600800050008001500080025042
:1010700000800350408004404480044008800440C5
:1010800070B50F490F4800F0E5FD0F4800F0E2FD94
:101090000E4E0F4D00242B196159DA68301C0A4B93
:1010A000143400F0D7FD782CF5D10A4800F0D2FDB9
:1010B00000F018FB011C084800F0CCFD70BDC046D4
:1010C000AE3A000078400000CA4000008A400000AC
:1010D0001C00001095400000B7400000F0B53C4BEC
:1010E0008BB01D68002D3AD03A4B02901B6801204E
:1010F0009B685DE001342378202BFBD0002B3AD095
:10110000B30008336A469C500136FF2D01D135E00B
:1011100001342378202B01D0002BF9D1202B02D1D0
:10112000002323700134012E1BD12A4F2A4B0722A2
:101130003B6001923D1C09E02B680298196800F0A1
:1011400003FE002808D02B6814332B60019B013B61
:101150000193002BF0D132E03B681D7901E0041CC3
:101160002E1C2378002B06D000230722B2425B41BD
:10117000DBB2002BBFD1002E1CD000E00025154CA7
:10118000022E05D10398154900F0DEFD002801D09C
:10119000AE420AD823681248D96800F05BFD236884
:1011A0001048196900F056FD04E02368F0B29B680E
:1011B00002A99847064B1B68002B07D103E0019852
:1011C000011CFFF75DFF084800F044FD0BB0F0BDC7
:1011D000D0020010D80200101C000010C440000013
:1011E000C6400000473B0000CD40000038B5041C5D
:1011F000154D0A2808D002D808281CD110E00D2867
:1012000002D07F2817D10BE02B6800221A700F48FC
:1012100000F020FD0E4C201CFFF760FF2C6012E058
:101220002A680B4B9A420ED90A48211C00F012FD85
:101230002B68013B06E00748211C00F00BFD2B68E2
:101240001C7001332B6038BDD4020010CA4000006E
:10125000D0010010D940000008B503E000F098FB71
:10126000FFF7C4FF00F0B6FB0028F7D108BD00006F
:1012700008B5034A034B04481A6000F0EBFC08BDB4
:10128000D0010010D4020010CD400000044B4021DA
:101290001A680A431A60034B01221A707047C0464D
:1012A00080800440DC02001070B50E4B061C1B78D9
:1012B0000D1C141C002B01D1FFF7E8FF013E022E8C
:1012C00003D8094BB600F35800E0084B1A68012C0C
:1012D00003D1AC4014431C6003E00124AC40A243A2
:1012E0001A6070BDDC0200105C41000000800050FC
:1012F00038B50F4B051C1B780C1C002B01D1FFF7D8
:10130000C5FF0020032D11D8281C012302F0C2FACA
:1013100002040608074A04E0074A02E0074A00E020
:10132000074A1068A3401840431E984138BDC04684
:10133000DC020010FC3F0050FC3F0150FC3F02501B
:10134000FC3F035070B50E4B061C1B780D1C141C83
:10135000002B01D1FFF79AFF013E022E03D8094B63
:10136000B600F35800E0084B1A68012C03D1AC40DA
:1013700014431C6003E00124AC40A2431A6070BD1A
:10138000DC02001068410000FC3F005038B5084BFB
:10139000041C1B780D1C002B01D1FFF777FF23687D
:1013A00018229343236023681D43256038BDC0463F
:1013B000DC0200101F234209184001238340181C3F
:1013C000014B9200D050704700E100E01F2342091A
:1013D000184001238340181C2032024B9200D05049
:1013E0007047C04600E100E0054B3F221A60054B04
:1013F00001221A60044B40211A688A431A60704720
:1014000024800440D88004403882044008B5044B4E
:1014100040211A688A431A60FFF7E6FF08BDC046FC
:101420003882044008B5154B1868FFF78DFD07207A
:10143000FFF7CCFF0820FFF7C9FF0A20FFF7C6FF20
:101440000C20FFF7C3FF0B20FFF7C0FF0920FFF7B9
:10145000BDFF0B4A0023136001210A4A4942116073
:10146000094A1360094A1360094B01221A60094BAB
:101470001A6801321A60C04608BDC0461800001044
:10148000048204400882044004C000403CC0004084
:1014900000C00040E002001008B5FFF717FC0A4842
:1014A0000021FFF773FF09480021FFF76FFF08488D
:1014B0000021FFF76BFF07480021FFF767FF064891
:1014C0000021FFF763FF08BD0840044000400440CE
:1014D000AC400440144004401C400440F8B5071CD4
:1014E0000C1C72B6FFF7D8FF434B1A68434B1A60C7
:1014F000002F01D0424B00E0424B434A04211360CD
:10150000424B434D1A680A431A6000232B609C42E9
:1015100018D00720FFF74EFF0820FFF74BFF0A20E7
:10152000FFF748FF0C20FFF745FF0B20FFF742FFB6
:10153000384B394A19680A401A602A68EC235B0163
:1015400013432B60002F4FD0344B354C35490026C8
:101550000E60201C1E60311CFFF718FF301C092193
:10156000321CFFF7A1FE301C0921321CFFF7EAFEF6
:101570002D4B8022196811431960236807218B4382
:101580002360236802210B4323607B00DB19990150
:101590005B189B002549DF19254B0F60032119605B
:1015A000244B2549186801401960196809200A432D
:1015B0001A60FFF7FFFE174A802311689B0019434A
:1015C00011602A68022113431C4A2B600123136017
:1015D0001B4A11601B4A13491360166013601068A0
:1015E0001842FCD001230B60174B012252421A60B3
:1015F00062B630BFF8BDC046388204403482044031
:10160000BF180000FF1800003082044010ED00E019
:1016100004820440008204407FE2FFFF0440014056
:101620006440044004C000408080044018C0004072
:1016300014C000403CC000400FF0FFFF7880044021
:1016400070800440748004400882044008B5FFF7AD
:1016500045FF08BD00B5064B1A6801321A601B68C9
:10166000013303D1034B1A6801321A6000BDC04632
:10167000E8020010E402001000B5074B98420AD8B7
:10168000064A00231360064A01381060054A1360B9
:10169000054B07221A6000BDFFFFFF00E8020010A3
:1016A00014E000E018E000E010E000E000B50C4AB3
:1016B0001368002800D10120C1438B4204D809E0FF
:1016C00011688142FCD301E0591C08181168994245
:1016D000F6D203E01168C91A8142FBD300BDC046AF
:1016E000E802001010B5064BFA211868054B890076
:1016F0001C6802F0E3F8044B5C43201810BDC046A0
:10170000E8020010E402001037894100034B012277
:101710001A60034B1A6801321A60704700C000401B
:10172000EC020010034B01221A60034B1A680132CD
:101730001A60704700000140F0020010034B0122C4
:101740001A60034B1A6801321A607047004001406A
:10175000F4020010034B01221A60034B1A68013295
:101760001A60704700800140F802001000B50028A0
:1017700003D1044B01221A6003E0012801D1024B7E
:10178000186000BD044001400480014000B50028FD
:1017900002D1044B186004E0012802D1024B002260
:1017A0001A6000BD044001400480014010B50028CB
:1017B0000FD1124B80221C68920022431A60104BFA
:1017C000032218600F4B19600F4B1A608022D2025F
:1017D00011E0012811D1094B80221868D200024380
:1017E0001A600A4B00221A60094B03221960094B48
:1017F0001A6080221203084B1A6010BD80800440DA
:10180000F40200101840014014400140F80200109A
:10181000188001401480014000E100E008B5184B39
:101820001A680E231340062B0DD1164B9E221B68FF
:10183000DBB2134204D0144A5360144B1B681EE001
:10184000D9071CD501E0042B05D1104B1868C0B294
:1018500000F0AFF813E00C2B06D10B4B8022596837
:1018600052000A435A600AE0022B08D1054B1A685D
:10187000054B910601D5002200E001229A6008BDC7
:101880000880004014800040FC02001000800040EE
:1018900000487047FC02001070B5294C294B80228B
:1018A0009203DA67061C0021201C902200F00AFA3D
:1018B0000023A360244B07251A68244CAA431A600E
:1018C0001968012211431960214B1968A943196055
:1018D0001968114319601F4B8021186849010143A1
:1018E00019601D4B1A608322226019681B4B18680F
:1018F00001F0E4FF311C000901F0E0FF1849030A80
:10190000184A0B60C0B2032310602360164B1D60A1
:10191000164B186860201C680440602CFBD101E065
:10192000146800E001201C680442F9D1044B012234
:101930001A700F4B802292031A6005230B6070BD52
:10194000FC02001004E100E0A44004400C800040D0
:10195000A84004408080044098800440C0040010E7
:101960000480004000800040088000401480004057
:1019700000E100E000B5044A202311681942FCD0C0
:10198000024B186000BDC04614800040008000403B
:1019900008B5FFF77DFF827B031C8218D07B9A7B02
:1019A0000132D2B29A7352B2002A01DA00229A733B
:1019B00008BD10B5041CFFF76BFF437BC318DC7335
:1019C000437B0133DBB243735BB2002B01DA0023AC
:1019D000437310BD08B5FFF75BFF827B437BD01AD2
:1019E000431E984108BD30B5002402E00570013463
:1019F00001301D5D002DF9D1121B131C02E0017096
:101A0000013B0130002BFADCD043C0170240A01884
:101A100030BDF8B5051C0F1C1E1C541E092B01D827
:101A200000240FE0181C0A2101F048FF221C031CAF
:101A3000391C281CFFF7EDFF041C2D1805E02F7042
:101A400001340135013A002AF9DC301C0A2101F089
:101A500079FF30312970601CF8BDF8B50C1CD9171E
:101A60005F18061C4F40551E092F12D9381C0A2139
:101A7000002B03DA01F022FF434202E001F01EFFD7
:101A8000031C211C2A1C301CFFF7E7FF041C35181F
:101A900013E0002B00DA951E002201E0B45401325D
:101AA000A91A0029FADCEC43E4172C403519002B65
:101AB00003DA2D232B7001340135381C0A2101F083
:101AC00041FF30312970601CF8BD73B5069E041CBF
:101AD0001D1C3009531E00280AD000901A1C201C1F
:101AE0002B1CFFF7F2FF241805E0217001300134B0
:101AF000013A002AF9DC0F231E40092E01D83036A6
:101B000004E0002D01D0373600E057362670013052
:101B100076BDF0B585B0041C0F1C002801D0002153
:101B2000017000256BE0252903D0217001320134BA
:101B300005E05178252904D12170023201340135A4
:101B40005DE0302903D001320292202101E002320F
:101B50000292029E9C4632782D3A50424241B6187B
:101B60000296002205E00A235A438218303AD2B284
:101B700001363078031C303B092BF4D90296AE189D
:101B80006346BE4201D97A1BD2B269280ED006D86C
:101B900063282CD0642809D058283ED119E0752834
:101BA0000AD078280FD0732837D11AE01E1D201CC8
:101BB0001B68FFF752FF04E01E1D201C1B68FFF787
:101BC00028FF331C17E01E1D1B68201C00930023F8
:101BD00004E01E1D1B68201C00930123FFF775FF06
:101BE000EFE71E1D201C1B68FFF7FDFEE9E71A68E2
:101BF000012022700433029A241801322D18117822
:101C0000BD4201D200298ED10023BD4201D22370F2
:101C100005E0013C2370013D01E001256D4205B066
:101C2000281CF0BD10B50C1C131C6421221CFFF7EE
:101C300070FF10BD00B5031C9BB00A1C01A8191C45
:101C4000FFF7F0FF632800DDFEE701A800F0A6F82B
:101C50001BB000BD0FB407B504A901C90191FFF77E
:101C6000E9FF03B008BC04B018470EB403B503AADB
:101C700002CA0192FFF7D6FF02B008BC03B01847B2
:101C800070B50323041C184205D10D1C041C194215
:101C900001D1934201D3002311E0131C40CD043B3A
:101CA00040C4032BFAD8141FA4080134A400032352
:101CB00009191A400419EEE7CD5CE554013393424B
:101CC000FAD170BD30B50B040D061D430D430B0258
:101CD0001D430323041C93420DD218420BD1131C45
:101CE000043B20C4032BFBD8141FA4080134A40018
:101CF00003231A400419002301E0E1540133934205
:101D0000FBD130BD00B5002300E00133C25C002AE6
:101D1000FBD1181C00BD00B5031C01E001310133EB
:101D20000A781A70002AF9D100BD30B5031C0024CE
:101D300006E01D5D085D281A05D10134002D02D092
:101D40009442F6D1002030BD00B502E00130002BF6
:101D500006D00A78037801319342F7D0981A00E050
:101D6000181C00BD08B5FFF753F90B4BFA21186892
:101D7000890001F0F1FDFFF77FFCFFF787FAFFF71D
:101D800045FB96200002FFF787FDFEF757FEFEF7A2
:101D900043FEFFF76DFA08BDC004001010B5041C27
:101DA00002E00134FFF7E6FD20780028F9D110BDEC
:101DB00030B5F8238A01DB0013404A05920E134325
:101DC000F8221202114019430A235943CA108318FA
:101DD0001C1CEB345D782478EA336C401B782402B9
:101DE0001C43835C201C5840072319400841800590
:101DF000800D30BD7047000008B5054B011C9842AE
:101E000001DD044BC1180448EA38FFF7D1FF08BDD3
:101E1000FF17000000F8FFFF7441000008B54018EC
:101E2000511A013101F0FAFD08BD08B58018891872
:101E30009A1A0132FFF724FF08BD000010B5CB004D
:101E4000591A074B0F22C9180023CC5C14400470A8
:101E5000CC5C0133240944700230072BF5D110BD4E
:101E60006005001010B5CB00591A064BC9180023A5
:101E70004278047812012243CA5401330230072BFE
:101E8000F6D110BD6005001030B5B14B87B0D96EEA
:101E9000B04D4A1E91416A46D175A96A1A1CC806FE
:101EA000400F0138062807D801F0F4FC040C1F127B
:101EB00017191C00022409E05A6E16329200D358FA
:101EC0001C1C15E05B6E16339B00D45800230FE0FA
:101ED0009B6DD46DA3420ADC0AE0022403E00C24CB
:101EE000032305E00D24231C02E00D24EEE70D245E
:101EF0002C6148111F2800D922E16A461732944903
:101F000001F0D2FC2000220028002A002D002F0022
:101F1000380040004400490051005F0067006F0036
:101F2000770085009300A200B400C300D500D30061
:101F3000E300E600E900F100010105010F011101D4
:101F400013011901081C00E08348191C221CFFF72B
:101F500065FFF5E08148F8E70A1C0E3203E07E4891
:101F600009E00A1C1C32081C111C1A1C231C01F05D
:101F7000CDF8E5E07948011C0E391A1C231CFFF747
:101F800054FFDDE07448011C0E31EEE70A1C1C32E0
:101F9000081C111CF1E70A6E1020002A00D00A204C
:101FA0000A1C0E3206E00A6E1020002A00D00A2019
:101FB0000A1C1C3200946C46173402900194081CD1
:101FC00051E001201070086E1022002844D00A222F
:101FD00042E00A6E1020002A00D00A200A1C0E32AD
:101FE0000EE001201070086E1022002855D00A2241
:101FF00053E00A6E1020002A00D00A200A1C1C326E
:1020000000946C46173402900194081C78E00A6E24
:102010001021002A00D00A21504A6846173001904A
:1020200002910094101C111C1DE00A6E1020002A61
:1020300000D00A20494A00946C46111C17340290C3
:102040001C390194101C0EE0096E01201070102242
:10205000002900D00A2241496846173001900292B7
:102060000094081C002201F05BF869E00A6E102061
:10207000002A00D00A20394A00946C46111C1734FB
:1020800002901C390194101C3AE0096E0120107076
:102090001022002900D00A223049684617300190EA
:1020A00002920094081C00222AE0012010700A6E9F
:1020B0001021002A00D00A21284A684617300190D2
:1020C00002910094101C00211AE0009222481CE0AA
:1020D0000092224819E00A6E1020002A00D00A203F
:1020E0000A1C1C3206E00A6E1020002A00D00A20CA
:1020F0000A1C0E3200946C461734029001940020A2
:1021000001F037F81CE00092081C002104E00D1CCF
:102110001C35081C0092291C1A1C231C01F084F891
:102120000EE0081C02E00C4800E00C48191C221CC0
:1021300001F093F804E0081C221C191C01F098F827
:102140006B46DA7D024B07B00120DA6630BDC0462F
:10215000C4040010600C0010D2040010E004001051
:1021600010B506490B1C88331A68141C1E34A400D1
:102170006050013203210A401A6010BDC4040010EF
:10218000054B0320191C88310A68013A02400A6095
:102190001E329200D0587047C4040010F8B5114D9B
:1021A0002C1C8C3420680130FFF726FE0E4B0122D8
:1021B000D8629F6AAB6E061C02409A4210D1830718
:1021C00003D420680230FFF7CBFFFF239B001E40A3
:1021D000B601BF10044B8C35374301222F60DA6003
:1021E0000220F8BDC4040010600C001030B50C4B88
:1021F0000C489A6A031C8C331C68D3059B0E91050E
:1022000000D5403B856E921001210A40AA4204D1BC
:10221000E3188C300360024BD960012030BDC0460A
:10222000600C0010C404001008B5084B5A1CD07F85
:102230009A1CD27F000112021043DA7F0333DB7F46
:1022400010431B031843FFF78BFF08BDC4040010A5
:1022500038B5FFF795FF064903230F22051C5C18CC
:102260001540013325770011072BF7D138BDC04643
:10227000C404001008B5FFF783FF034B01228C3321
:102280001860024BDA6008BDC4040010600C001036
:1022900010B5064CA36E002B06D0FFF771FF044B60
:1022A0008C3401222060DA6010BDC046C4040010E6
:1022B000600C001010B5064CA36E002B06D1FFF782
:1022C0005FFF044B8C3401222060DA6010BDC046F1
:1022D000C4040010600C001008B5124B1B68002BE2
:1022E00000D09847104B5A69002A15DD012A07D102
:1022F000DA69002A04D09A610022DA610A225A615E
:102300005B690322191C91430A1E02D0074A01216E
:10231000D166054A013B5361044B90331A68024B66
:102320005A6208BD8C030010600C0010C404001039
:1023300000B5064B5A69002A07DD9A690F21044B44
:102340001140D97712110133DA7700BD600C00100B
:10235000C4040010044B597F9A7F090112020A43FA
:10236000197F0A435A677047C404001030B50B1C2C
:10237000093B012B0FD8084A00239C18257FC45C19
:10238000A54205D0054B08395A681143596002E04F
:1023900001330E2BF1D130BDC4040010600C0010CD
:1023A00008B508290DD0192913D1427808231A42FB
:1023B00002D00022027002E00F2303700723437053
:1023C00005E000231A1CC25401330E2BFBD1FFF78A
:1023D00049FD08BD1FB50E4B5C6F002802D00F22CF
:1023E000944304435C67FF2C10DC6846211CFFF714
:1023F00025FD6846211CFFF7D3FF054A00236C46E4
:10240000185D9918013308770E2BF8D11FBDC0460F
:10241000C404001030B5124C0F23656F85B09D4386
:1024200005436567082D19D0FF2D17DC6846291C68
:10243000FFF704FD6846291CFFF798FF00231A19CF
:10244000127F69465A5401330E2BF8D16846291C75
:10245000FFF7A6FF6846291CFFF704FD05B030BD55
:10246000C40400101FB50F4C616F082918D0FF2954
:1024700016DC6846FFF7E2FC616F6846FFF776FFFF
:1024800000231A19127F69465A5401330E2BF8D1D2
:10249000616F6846FFF784FF616F6846FFF7E2FCF3
:1024A0001FBDC046C404001010B50D4C631CD87F7E
:1024B000A31CDB7F00011B021843E37F1843E31CCE
:1024C000DB7F1B031843FFF797FC0F23021C1A4006
:1024D00022770211134000126377A07710BDC04627
:1024E000C4040010044B5A6E16329200D258121ACD
:1024F00051424A41DA667047C404001000B5064BE9
:102500005A6E16329200D1580139D150002901DAA1
:102510000D21D15000BDC046C404001000B5064BCB
:102520005A6E16329200D1580131D1500E2901D184
:102530000021D15000BDC046C404001000B5094BB5
:102540005A6E16329200D2580D2A03D11A1C293223
:10255000127805E09A18507F117F0001021C0A438F
:102560005A6500BDC404001010B5084B0F245A6E04
:1025700016329200D1585A6D581814400131047720
:102580000D2902DC5B1812111A7710BDC40400106B
:1025900030B50F4B5A6E596D16329200D2580D2A33
:1025A00007D11C1C29342478F020084020435865AA
:1025B00007E09818447F057F24012C435C650B11CC
:1025C0004377034B9A180F231940117730BDC0464B
:1025D000C404001008B504480022011C1C390D2356
:1025E000FFF723FC08BDC046FC04001008B50448F2
:1025F0000022011C1C310D23FFF717FC08BDC0464B
:10260000E004001008B504480022011C1C310D2311
:1026100000F07CFD08BDC046E004001008B5044889
:102620000022011C0E390D23FFF7FFFB08BDC04639
:10263000EE04001008B504480022011C0E310D23E1
:10264000FFF7F3FB08BDC046E004001008B50448DE
:102650000022011C0E310D2300F058FD08BDC046BC
:10266000E00400100C4A0023111C46310B70111CB1
:1026700047310B70111C48310B70111C49310B7024
:10268000111C4A310B70111C4B310B70111C4C3159
:102690004D320B7013707047C404001000B5074A28
:1026A000011C042300208A1804E0D118463109785F
:1026B00040000843013BF8D200BDC046C4040010EE
:1026C00030B5074A00238918012206E0CC18051C02
:1026D00046341540257040100133042BF6D130BD2F
:1026E000C404001038B50020FFF7D8FF084C051CC3
:1026F0000021207FFFF7E4FF25770420FFF7CEFFBE
:102700000421051C607FFFF7DBFF657738BDC046FD
:10271000C404001010B50020FFF7C0FF034C207761
:102720000420FFF7BBFF607710BDC046C404001053
:1027300010B5054C0021207FFFF7C2FF607F042108
:10274000FFF7BEFF10BDC046C404001010B5094C11
:10275000231C8C3318680130FFF74EFB064B021C1C
:10276000D8620F231A4022770211134000126377B8
:10277000A07710BDC4040010600C001010B5094C07
:102780000021201C0D22FFF749FB201C0E300021E8
:102790000D22FFF743FB201C1C3000210D22FFF708
:1027A0003DFB10BDC404001010B50C4B00211A1CD9
:1027B000187F1C7801312043187701330E29F7D197
:1027C000936E002B08D0064B1B690D2B04D1137F91
:1027D000111C29310B70537310BDC046C404001086
:1027E000600C001010B50C4B00211A1C1C7F1878CF
:1027F00001312040187701330E29F7D1936E002B59
:1028000008D0064B1B690D2B04D1137F111C2931F5
:102810000B70537310BDC046C4040010600C001050
:102820007FB500230C4A0D251C1C1118097F0130AF
:102830006E469955C60F8542664176420133111C9A
:1028400030400E2BF1D100236C46185DCA180133BD
:1028500010770E2BF8D17FBDC404001010B5074BC4
:102860005A6E16329200D1585C1801392077D15037
:10287000002901DA0D21D15010BDC046C40400105A
:10288000034A0023111C943198320B601360704787
:10289000C4040010034B012194331A684A401A60A3
:1028A0007047C046C4040010044A002313678C32EA
:1028B0001360034B0122DA607047C046C404001065
:1028C000600C001008B59A4B0F20996A994A8B103A
:1028D00018408911013852560E2800D9C1E000F085
:1028E000D9FF08111A2327C02EC0C037C0C0C03B73
:1028F0003F00002A00DAB4E08F4B9A1840320023E0
:102900009371A9E0002A00DAABE08B4B01209A1802
:1029100040329071A4E0002A00DAA2E0864B9A18B7
:1029200040329279DA6697E0081CFFF797FF93E050
:10293000002A00DA95E0101CFFF7D4FD8CE0002A95
:1029400000DA8EE07C4B596E16318900CA5083E064
:10295000081CFFF75FFD7FE0081CFFF73BFD7BE0F5
:10296000002A00DA7DE0101CFFF75AFF74E0724B7A
:1029700001209833186073E0FFF7E0FD6CE0FFF78B
:1029800093FF69E0FFF726FE66E0FFF7EDFD63E0E9
:10299000694B00225A665FE0FFF728FE5CE0FFF714
:1029A000F7FD59E0644B0120586659E0FFF72AFE15
:1029B00052E0FFF7CBFE022052E0FFF72FFE4BE084
:1029C000FFF732FC48E0FFF735FE45E0FFF7D6FEA3
:1029D00042E0FFF73DFC3FE0FFF738FE3CE0FFF749
:1029E000A7FC39E0544B00221A6635E0FFF7B2FC31
:1029F00032E0514B0120186632E0FFF741FF2BE037
:102A0000FFF730FD28E0FFF745FF25E0FFF74CFD1D
:102A100022E0FFF78DFE1FE0FFF73AFC1CE0FFF716
:102A2000C3FE19E0FFF776FE16E0FFF743FC13E064
:102A3000FFF7D8FE10E0FFF715FE0DE0FFF74CFCA6
:102A40000AE0FFF75BFD07E0FFF74CFE04E0FFF74D
:102A500065FD01E0FFF70EFC012001E0012040428E
:102A600008BD982BBED03EDC382B9BD01DDC1C2B28
:102A700000D187E70CDC0C2B00D178E702DC002BBF
:102A8000EAD0EBE7162B00D176E7182BE6D176E7F4
:102A9000282B00D17CE702DC262BDFD175E72C2B1D
:102AA00000D179E7362BD9D179E7662B00D18AE7B7
:102AB0000CDC4C2B00D17CE702DC3C2BCED175E743
:102AC000562B00D179E75C2BC8D179E76C2B00D16C
:102AD0007FE702DC682BC1D178E7762B00D17BE75A
:102AE000882BBBD17BE7E62B00D19BE726DCC82BEC
:102AF00000D188E70CDCA82B00D17AE702DC9C2B04
:102B0000ACD173E7B82B00D177E7BC2BA6D177E720
:102B1000D62B00D17DE703DCCC2B00D09EE775E7F8
:102B2000D82B00D178E7DC2B00D097E777E7C046B9
:102B3000600C0010747D0000C4040010F32B00D161
:102B40007CE70EDCEC2B00D172E703DCE82B00D035
:102B500084E76AE7F12B00D16DE7F22B00D07DE727
:102B60007AE7F62B00D16FE703DCF52B00D075E791
:102B700067E7F72B00D16AE7F82B00D06EE769E72B
:102B800038B5184C231C8C331868FFF735F9E26E02
:102B9000154BA2660022E266DA6003229862251CC9
:102BA00010401C1C022809D090420AD0012802D0F3
:102BB000FFF788FE07E0FFF7F1FA04E0FFF764F99A
:102BC00001E0FFF713FB002807DDE368002B04D1C9
:102BD0002B1C8C331A6812181A6090352B681B183E
:102BE0002B6038BDC4040010600C0010034B0122A0
:102BF000DA660F229A775A771A777047C404001062
:102C000010B5054C0549201C00F008FFFFF7EEFF4A
:102C10000123636610BDC046C40400109C07000079
:102C200000B5074B00201B680F2B08D1054B1A7805
:102C3000824204D11868044B1840431E984100BDDD
:102C400094000010C404001000FFFF0038B5164BBC
:102C50001A1C98321268002A04D0144B1D680123F4
:102C60001D4001E094331D68114CA3689D4202D1C0
:102C70006268002A16D0002D02D1002B0AD111E083
:102C80000C4B1B68002B02D06168281C984700235E
:102C9000636006E0074B1B68002B02D0281C291C30
:102CA0009847A56038BDC046C4040010AC030010AE
:102CB000600C0010A403001013B5002300930193CF
:102CC000244B1B68002B02D0684601A99847224973
:102CD000009B0878214A00280CD0002B02D0022348
:102CE000137035E01378013BDBB21370002B2FD14A
:102CF0000B7009E0002B0CD11378002B28D0013B7E
:102D0000DBB21370002B23D1154A1360154A1360F0
:102D10001EE014490968581A44426041400010708E
:102D200011484469021C002C04D08B4202D10A23B2
:102D300043610DE000290BD10A2151610199936192
:102D4000D161084A1360064B02221960034B1A70C6
:102D500013BDC04694030010B00300109803001088
:102D6000940C0010900C0010600C001008B5FFF7D8
:102D7000A3FF08BD30B50A4D049C286009480160D6
:102D800009490A60094A1360094B039A1A60094B02
:102D9000094A1C60094B1C60094B1A6030BDC046D3
:102DA000A403001094030010A00300109C03001063
:102DB00090030010940000106D2D0000600C0010B6
:102DC0008C03001008B5084B084A196812688A1A63
:102DD0001A6006D5FA2252001A60054B1A680132B1
:102DE0001A60FFF733FF08BD980000109003001031
:102DF000AC030010F7B50E1C0E21051C019200F06B
:102E00000DFE1A4B03240C279E420FDD09236B7322
:102E100001232B7328E0301C0A2100F0F3FD301C45
:102E200029550A2100F098FD0134061C002E06D019
:102E3000E30F0022A7425341DBB29342EBD1019A48
:102E4000A31A033B2B70621B2B1C01E0195D597305
:102E5000013BD1180229F9D10F231C1B002301E0EB
:102E6000013C2B55032CFBDCF7BDC046FFC99A3B48
:102E7000F8B5104B01221A700F4B0222041C1A7075
:102E80000E4E0F4D0FE0196891420FD01B682B605A
:102E9000FFF798FFFFF710FF002C04D0013C002C37
:102EA00001D13C7005E033682A68024F3978002967
:102EB000E9D1F8BDB0030010980300109C03001086
:102EC000A8030010F7B51C4D9B235B000E1C1B4A8A
:102ED000E95C1B4BAC5CEB5C002902D00F22144078
:102EE00002E08021072449009A225200AF5C154A73
:102EF000CB1AAA5C3435BA1A80277F00791A009160
:102F000007210C1B013210490194FEF7AEFE00238D
:102F10000E4F33704124FF35301CFEF7F3FE2A7844
:102F20006B783018D31A391C221C0134FEF79DFE31
:102F3000013D462CF0D1F7BDC4040010370100005C
:102F40002F01000035010000847D0000917D00000C
:102F500070B5314B314C1A1C9432126890B0A0619C
:102F6000E161002A17D118280BD1C32909D12C4AB5
:102F700012680F2A05D1181C38300E21162200F0D5
:102F8000B1F8A369182B04D1E369332B01D100F008
:102F900053F8FFF72BFE0A231F4D6361214E0123D7
:102FA0002B678C35FFF7ECFD002801DAFDF75AF9A5
:102FB0002B68B34203D01C4A934214D104E0FFF7BC
:102FC00045FEFDF784F80EE0184C2368002B0AD06C
:102FD000684608A9FFF776FF2368684608A998475E
:102FE0002B6827332B60124B1A68124B1068196834
:102FF000884205D012681A60FFF7E4FEFFF75CFE16
:10300000054B1C6F002CCDD1FFF720FE201CFFF7D5
:103010002FFF10B070BDC046C4040010600C00103B
:1030200094000010790D00003E270000A00300105E
:103030009C030010A803001070B5254C00202368E5
:103040001D68FFF715FF23681A689542FCD01E68BB
:10305000FFF7CCFD1F4B0A221F4C5A6118229A61C0
:103060001522DA61231C903300221A60FFF7BEFD9F
:103070002D3601232367FF36154C184D0AE0FFF764
:103080007FFD23682A681968914203D01B682B6072
:10309000FFF798FE23681B689E42F0D10E4C182063
:1030A000231C903300211D68FFF752FF0C4B281C96
:1030B000196800F051FC3834011C0422201CFFF771
:1030C00099FE044B18229A610022281CDA6170BD17
:1030D0009C030010600C0010C4040010A803001032
:1030E00090030010F0B501240DE005780B1C25407D
:1030F00006E0C65CED0077083D43C554351C25400D
:10310000013BF6D5013A002AEFDCF0BD30B504E012
:10311000845C8D5C85548C5401329A42F8DD30BD5C
:10312000F7B5099D0AAC2678089F2C7894461D1C9B
:10313000002A0DD118E063465B5D4A5DD218131971
:1031400001920024B34201DB9B1B0124435501354E
:10315000BD42F0DD0AE0CA5C12190024B24201DB74
:10316000921B0124C2540133BB42F4DD099B1C7045
:10317000F7BDF7B5099E0AAC2778089D347800287A
:103180002FD000292AD01E1C9446002A0ED1013FC0
:1031900018E063469B5D8A5DD21A131B00240192DE
:1031A000A34201DADB19012483550136AE42F0DD7A
:1031B00037E0CA5C121B0024561C01D13A1C0124C2
:1031C000C2540133AB42F4DD2BE0D15C49420C1B0D
:1031D000211E01D0E1190124C1540133AB42F4DDB9
:1031E0001FE000291BD0181C002A06D10EE00E5C3F
:1031F000135C0130F31A1C1BE40FA842F7DD10E04A
:10320000CA5C0133141B013462425441AB42F7DD06
:1032100007E0D15C013349420C1B611E8C41AB427B
:10322000F7DD099A1470F7BD70B5049D01242C7068
:10323000141C002905D10BE0065D0A5D96420BD1F6
:1032400001349C42F8DD05E0815C002904D10132A3
:103250009A42F9DD00232B7070BD00B503E04318DE
:103260005B78435401319142F9DB0023435400BDA4
:1032700000B504E08318013B1B788354013A8A426D
:10328000F8DC0023835400BDF0B5114B1A785B784D
:10329000825C1A4000D040220E4C0F49231C261C91
:1032A00004C32C3600221A6001240A1C123117783C
:1032B0005578C75D3D4202D01F6827431F60023228
:1032C00064008A42F3D10433B342EBD10020F0BD55
:1032D00091010010280E0010DD00001030B51223FF
:1032E0004B43334A0131D3188A0051181A785C785D
:1032F000825C144204D02F4A5F2452189470547098
:103300009A78DC78825C144204D02A4A7C245218D1
:10331000533214701A795C79825C144204D0254AC5
:103320007C245218A33214709A79DC79825C14429E
:1033300007D0204C5F226418251CA235A1342A70C6
:1033400022701A7A5C7A825C144204D0194A7C2476
:103350005218A03214709A7ADC7A825C144204D03B
:10336000144A7C245218503214701A7B5C7B825CA5
:10337000144207D00F4C5F226418251C523551347B
:103380002A7022709A7BDC7B825C144204D0094A4A
:103390002E245218A43214701A7C5B7C825C134277
:1033A00004D0044B5918F43127230B70002030BD92
:1033B000DD000010980C0010F8B52D4C071C0025FE
:1033C000201C20214F22FEF77DFC002D04D0221C62
:1033D0007C23393223701370231C4F3300210135B5
:1033E00019705034052DEBD1214B2D22181C38308B
:1033F0000270181C37300270A1209A705A70400079
:103400005F221A541B481A54A320400019541A4929
:1034100008784978385C014204D0191C5331523382
:103420000A701A700024211C381C0134FFF756FF63
:103430000A2CF8D1114D124E00242B786A78FB5CCF
:103440001A4201D0315905E03059FEF75BFC0D49B5
:10345000091A0A310C48043400F0EAFA0235242C27
:10346000EBD10A49084800F0E3FA0520F8BDC04650
:10347000980C001041010000910100109C00001008
:10348000B000001093010010D80D0010997D0000CD
:10349000F0B585B001900027FDF7BEFA6A4C3E1CDE
:1034A0006A4A7542754113687D19002B00D1D5E039
:1034B000002303AA537023687F210B405C2B00D1AB
:1034C0009EE02BDC382B00D192E013DC072B6CD074
:1034D00006DC022B00D19BE0062B00D0BEE043E0CF
:1034E000212B00D188E0232B00D18FE01C2B00D0B2
:1034F000B4E089E04F2B4ED007DC3F2B64D0402B4B
:1035000064D0392B00D0A9E066E0542B00D17DE0D7
:103510005B2B3ED0502B00D0A0E06FE0732B69D026
:1035200010DC662B39D005DC5E2B57D0622B00D027
:1035300094E067E06F2B3CD0712B53D06D2B00D003
:103540008CE02CE0792B4BD007DC762B4ED0772B00
:103550003ED0742B00D081E046E07D2B23D07F2B22
:1035600025D07C2B7AD135E031231370022E51DD2A
:10357000231C083B1A687F231A40542A07D0032EC5
:1035800048D0221C0C3A12681340542B42D14C22D2
:1035900006E032233DE033233BE0342339E035229B
:1035A00003AB1A7036E0362333E0372331E038239B
:1035B0002FE039231370062E2CDD231F1B684722B2
:1035C0001940232926D1EBE7302322E02D2320E0E8
:1035D00041231EE04222E3E74322E1E7442318E0CF
:1035E000452316E0462314E04822D9E7482310E09B
:1035F0004C230EE050230CE052230AE05222CFE786
:103600004F2306E0552304E05522C9E74E2300E08E
:10361000492313700E4B03A8291C0022FDF7F0FA72
:1036200023681A0605D5E91D0A480022084BFDF754
:10363000E7FA2368DA0572D5E91D07480022044B32
:10364000FDF7DEFA6BE0C046280E0010A001001066
:103650000000001005410000A17D00002368012248
:10366000134206D0A818C0B2002107220223FDF79A
:1036700051FA23680222134205D0A81DC0B20021CE
:103680000623FDF747FA236804210B4205D0A81D45
:10369000C0B202220623FDF73DFA236808210B423F
:1036A00005D0681CC0B207220223FDF733FA236855
:1036B000DA0606D5681CC0B2042102220623FDF7F3
:1036C00029FA23689A0606D5681CC0B20021022296
:1036D0000623FDF71FFA23685A0606D5681CC0B2F8
:1036E000042107220223FDF715FA23681A0607D5DD
:1036F000281C09300222C0B20821131CFDF70AFA67
:103700002368DA050BD5EDB2281C0930C0B20B21B5
:103710000A35FDF7E9F9E8B20A21FDF7E5F90136C6
:1037200004340C370B2E00D0BAE6114B1B68002B6B
:1037300005D01048002109220F4BFDF761FA0F4D0B
:103740000F4E104F0024019A2B78D35C6A781A42EE
:1037500006D0A3009859E15D0922074BFDF750FA06
:1037600001340235092CEED1FDF760F905B0F0BD4A
:10377000CC010010A37D00000C0000109C00001084
:10378000A4010010D400001038B5FFF749FA002852
:1037900014D006240321201C00F0DEF80321C5B25A
:1037A000201C00F02FF9281CC9B2FDF79DF9092C47
:1037B00001D10B24EEE701340E2CEBDDFDF736F9D9
:1037C00038BD000070B5041CFFF75EFD201CFFF73C
:1037D0005FFE0A4B1B78002B0ED0201CFFF7ECFD80
:1037E000074CC8235B00074EE518211C301C5034E1
:1037F000FEF730FAAC42F8D170BDC046B1030010FC
:10380000980C0010473B000000B589B000280ED08E
:10381000FDF7CDF801A80921FEF710FB684612302C
:103820000A21FEF70BFB01A8FFF7CCFF08E0FDF72C
:10383000C6F8044B1B78002B02D00348FEF70AFAA7
:1038400009B000BDB1030010A57D000000B5FEE782
:1038500000B5FEE708B50A4B0A4A0B4903E01078A9
:103860000132187001338B42F9D3084B084900220A
:1038700001E01A7001338B42FBD3FCF765FEFEE7D3
:1038800000000010FE7D0000C8010010C8010010FB
:10389000540E001002B4714649084900095C490001
:1038A0008E4402BC7047C04603B4714649084000CC
:1038B0004900095A49008E4403BC7047002934D09E
:1038C0000123002210B488422CD301242407A142F2
:1038D00004D2814202D209011B01F8E7E400A142AF
:1038E00004D2814202D249005B00F8E7884201D34A
:1038F000401A1A434C08A04202D3001B5C08224322
:103900008C08A04202D3001B9C082243CC08A04292
:1039100002D3001BDC082243002803D01B0901D07E
:103920000909E3E7101C10BC7047002801D00020F3
:10393000C04307B4024802A14018029003BDC0462C
:10394000D90000000029F0D003B5FFF7B9FF0EBC85
:103950004243891A1847C046002941D010B4041CBC
:103960004C40A44601230022002900D549420028EA
:1039700000D5404288422CD301242407A14204D21E
:10398000814202D209011B01F8E7E400A14204D2FE
:10399000814202D249005B00F8E7884201D3401A15
:1039A0001A434C08A04202D3001B5C0822438C0837
:1039B000A04202D3001B9C082243CC08A04202D3A1
:1039C000001BDC082243002803D01B0901D0090991
:1039D000E3E7101C6446002C00D5404210BC704741
:1039E000002806D003DB0020C043400801E080200F
:1039F000000607B4024802A14018029003BDC04669
:103A0000190000000029EBD003B5FFF7A7FF0EBC9B
:103A10004243891A1847C0467047C04600B500297E
:103A200005D000230139037001300029FAD100BD0F
:103A3000F8B5041CA30719D1231C04CB0F4D104E5D
:103A400050199043021C201C32420FD1181C0B4FFE
:103A500004CBD5199543354208D1181C074F04CB28
:103A6000D51995433542F1D000E001300378002BA1
:103A7000FBD1FEF750F9201CF8BDC046FFFEFEFE4C
:103A8000808080802578000D0A413A200020202582
:103A9000633A20000D0A4D3A20002020473A2025A5
:103AA0003032780D0A0025732025730D0A00444D2D
:103AB00031355F4D31420053455249414C20434F0F
:103AC0004E534F4C45007265616479000D0A42798E
:103AD000652E2E2E0D0A004C43443A2530326920C3
:103AE0002D202569002573202573202025694D4848
:103AF0005A0056313300202025692E25303369566F
:103B0000007475726E6564206F6E004241543A20F5
:103B100025696D560D0A000D0A25303278202000E7
:103B200057616974696E6720666F722064617461A1
:103B30002E2E2E0D0A00426164206D6F64656C0D9F
:103B40000A00526561642025730D0A004F4B004640
:103B500041494C4544006F6666004C43442064650F
:103B60006275672025730D0A00000000005C000CE0
:103B7000000C7C287C7C447C241048285408000CD1
:103B800000384400443800201008103810804000ED
:103B9000101010004000201008384438007C0064E9
:103BA00054484454281C107C4C5424385420047429
:103BB0000C28542808543800500080500010284425
:103BC000282828442810045408384C5C7814787C41
:103BD00054283844447C44387C54447C140438448D
:103BE000347C107C007C0020403C7C106C7C40408D
:103BF0007C087C7C047C7C447C7C14083844787C85
:103C00001468485424047C047C407C3C403C7C2068
:103C10007C6C106C1C601C64544C7C4400081020AC
:103C2000447C000804088080800408007844780000
:103C300007080400000000BF01BF010905000007DC
:103C4000000700070007130A00002000E400FC0042
:103C50003F00E700FC003F002700040F0800000CB5
:103C6000011E01FF03FF032201E201C2190D000042
:103C70000E001F0011019101FF007E00FC00FE01FB
:103C800013011101F001E0140A0000EE00FF011120
:103C9000011101BF01EE00E0013001100105030038
:103CA000000F000F0A050000F800FE0307070104DB
:103CB0000B060000000001040707FE03F80F0800D0
:103CC0000000000A000E001F001F000E000A11096C
:103CD0000000100010001000FE00FE001000100098
:103CE00010080400000004800780030D0700001086
:103CF0000010001000100010001008040000000068
:103D0000800180010D07000C000FC003F0003C0093
:103D10000F00030F080000FE00FF01010101010177
:103D200001FF01FE10080000000002010201FF0176
:103D3000FF0100010001100800008601C7016101B8
:103D4000210131011F010E010F08000082008301D3
:103D5000110111011101FF01EE11090000300038BD
:103D6000002C002600FF01FF012000200F080000AA
:103D700080009F011F0111011101F101E10F0800F5
:103D800000FC00FE010B0109010901F901F00F0817
:103D9000000001000100C101F1013D000F00030F0F
:103DA000080000EE00FF01110111011101FF01EEF9
:103DB0000F0800001E003F0121012101A101FF00A9
:103DC0007E0804000000008C018C01080400000043
:103DD000048C078C0312090000200070005000D8EA
:103DE0000088008C0104010401110900004800480A
:103DF00000480048004800480048004811090000F9
:103E0000040104018C018800D80050007000200DCE
:103E100007000002000300B101B9010F0006190DEF
:103E20000000F800FC010603FB06FD05050505057D
:103E3000FD05FF050601FC01F8120900008001F0F4
:103E4000017C004F004F007C00F00180010F080052
:103E500000FF01FF01110111011F01FE01E0110925
:103E600000007C00FE0083010101010101018301CA
:103E70008211090000FF01FF01010101010101831D
:103E800001FE007C10080000FF01FF01110111017B
:103E90001101110111010F080000FF01FF011100C4
:103EA00011001100110001120900007C00FE0083C6
:103EB00001010121012101E301E20112090000FFDA
:103EC00001FF011000100010001000FF01FF010AA7
:103ED0000500000101FF01FF0101010B06000100C7
:103EE0000101010101FF01FF10080000FF01FF01B6
:103EF00038006C00C6008301010110080000FF01BA
:103F0000FF0100010001000100010001160B00008B
:103F1000FF01FF010F003C00F000F0003C000F002B
:103F2000FF01FF0112090000FF01FF010F001C004B
:103F30007000E001FF01FF01130A00007C00FE0099
:103F400083010101010101018301FE007C0F0800D2
:103F500000FF01FF012100210021003F001E140A83
:103F600000007C00FE0083010101010101038307C1
:103F7000FE047C0412090000FF01FF012100210062
:103F80007100DF008E010001110900008E009F0109
:103F90001101110111011101F301E21109000001E8
:103FA0000001000100FF01FF0101000100011109F2
:103FB00000007F00FF008001000100018001FF0080
:103FC0007F1109000007001F007800E001E0017880
:103FD000001F0007190D00000F007F00F001E00135
:103FE0007C001F001F007C00E001F0017F000F1229
:103FF0000900008301C7016C00380038006C00C75D
:1040000001830111090000010007001E00F801F8FA
:10401000011E00070001120900008101C1016101B8
:10402000310119010D010701030100070008000A11
:104030000100181110133831303378717073C8C112
:10404000C0C38881808384848782C5C4C7C27574D5
:10405000777235343732151417120207020802013D
:1040600000030109030402040205030500062024DD
:10407000282C383C4044484C4669726D7761726523
:104080002025735F5631330D0A00252D3130732002
:1040900025732573000D0A5479706520273C636FE2
:1040A0006D6D616E643E203F2720666F72207061E7
:1040B00072616D730D0A00557074696D6520257508
:1040C000730D0A003F0025730D0A0D0A00564F5963
:1040D00041474552203E3E200025630048656C70F4
:1040E000004E6F20706172616D73004B65792070B6
:1040F00072657373003C6B6579313E203C6B65796A
:10410000323E202E2E2E0044756D70206D656D6F31
:104110007279006C004C6F6164206D656D6F72790F
:10412000007400546F67676C6520646973706C611C
:1041300079206F757470757420746F20636F6E735F
:104140006F6C650062005265616420626174746521
:10415000727920766F6C7461676500000080015091
:104160000080025000800350FC3F0150FC3F025091
:10417000FC3F0350EAB820226077373A812A339413
:10418000CFF87C5798A0396BFCF718377F727EBE4A
:10419000AC0F12A47073C61C0C817246B11A35D2D2
:1041A0007022707C0D6E3C2154F4FAD5EF09B513E2
:1041B000D698FF88360AB8E98A7B197E279230663E
:1041C000871181362D00882542BA65DA4D93BCF9F6
:1041D00087C900E7720FBCF17B7530EC72B27204D4
:1041E000D1796C11FC24188D5D48719E680C2F3EAE
:1041F000805D5508C121C9F10CDBCB1700BDB0D7DC
:10420000049ACF060BE482CFCA6E46445D404D92BD
:104210005EA4D2AD14F3AE437B67EB32A10F57E936
:10422000306DD7637AF2F236A2D11D7B200622CC04
:10423000FE6910607B74B5C8FD8DF27985BA4BD2EA
:104240008DCD43E4235B0CA07398106E8556849744
:104250001F5D4DBE3ADCAC903A2670BE4DD5AB2406
:104260009881AE730FB84C2E10E18E98EB0E843A05
:104270008C4C49A3B9C53E5417CE9FFD145C310B3D
:1042800044184C31304204F20433FAB146A61D3EC4
:10429000BC798D90F845CECA549F594CDC4A1EDF3C
:1042A00041CA20590A457777AB4DA6DC58853806B8
:1042B000B121EDC18B1C0C6347E225038FBEA29593
:1042C0002938816A21F77B98514899705FED64AB7A
:1042D0003489887CAF5692E9738E01E6688564DF85
:1042E00033FDD82B134ABD8955FBF1CEDABCC9FF8B
:1042F00096FF27960462E3F673F462841EA97BA5F9
:104300005ECEE20FE483E32F50AC21B7583AF76852
:1043100077BC43C5DA9A215109558BBC3896613177
:10432000ACC4BD6D3273DF3AB3085E38712203CB83
:104330008C8BA7A012E2A454B5A54AEE4EAF3BB9B0
:1043400030FFDAA8C948D73D2A4F14847AFE96C8B0
:104350003E42E61DCF18A02A3C349C480985B3F59F
:10436000F5C53EC1866D5D4325910139D95228734B
:104370000DEEC5B673A2B71FA4FCB67A35B8F1F737
:1043800004EB9BF3821250DEDF2AB5240454C07C78
:10439000274628989BFBD40A25B5BCB08F42A6249B
:1043A0003C913EB885A7C5B66A873BED8F40EDA925
:1043B000FD94405CEBF8D5ECC3314157CFAC75941C
:1043C0009FD93F8E00D8D925844BD8094E71239AA6
:1043D0003D3545CEC346A74CE959AD26C6463457B0
:1043E000BFBA936A990AA748B1A263FEFC84179DDD
:1043F0008E3F4985008E09FC6BD0CD6DE9A8E5CADA
:104400009C7A1C66077351B0ADABE9F5087BC34BD2
:10441000D81A467F5DAB620AF6C0889836F4A06968
:10442000E31A1925548EC423D6D788C39EA70D0F2F
:10443000C71FCF912E37411FB2FB9F8F6697F402A3
:10444000D1EA309A90700885B6BB61020F8692B3AC
:104450003B157367670BC178D7E9F824E0FD7B66ED
:104460005B3E0CFCA76F125EF116EF1AA83DB2DF9F
:10447000242E496EA5A0F16F30F8222818599F6E9E
:104480004873C4AB8F9E7AAF7423B44529E8C649FC
:1044900035FBE2AC559D8293D3898FB6962EC0A88A
:1044A000B452CBE2E19563C1210EDAF48CBE11A3C4
:1044B0001C14F54FBF23EA8781EEF7E5C21A01CD40
:1044C0009C028519727CD68AF363C962161E515B01
:1044D00047F3525E7498AE048A3CA74C0B8F293880
:1044E000B06F7F28C9F6B1EFC5FA27BBAD3FCB5FF0
:1044F00065E4CA7B67A51E3CC0D22D42634F39E9F3
:104500008317B6F0E9929CDF988DC71A2DF71483B4
:10451000B153048398131FA173BFD4593FF138726C
:104520001D2651F5AD8FDE747C19E9BEB82AD16C19
:1045300007663749E54366B092E90B3DE53E3A51DF
:104540000CF0DCFF9DD6E9CFB7FE9E920EFABE5F5F
:10455000D653FFD2091EC0A7513A0A2ED45E0F6B64
:10456000CEF711087D7524698DE8C7EFBECB59C918
:1045700083C4D50CE7B8660857FFF9CBB19C0BBED6
:104580008A504B0B2A37A9F8B0142191F287EA1907
:1045900010D119DD7AB6D5A3E23B49CEAF298EE81A
:1045A0001B8209DEF6C2DE3CFBBF9602A3832231EA
:1045B000A36A700FD9AEE6925ED1B48EC95C747FE7
:1045C000BADC7DF5AA74F3A7CF641182B1210E2A5B
:1045D000E25043B825BBAD2CD32FB874168A3B6686
:1045E0005A350724B7B7E64E3FD9789EEF9654BFA9
:1045F000CADBB3BD4585B6146F47B153D8D4175A3B
:10460000E4F95E777407F24AD8B2073249E1ACFBAD
:10461000423B9C01BBF2809CEB1A8EFEFCF15F9F3B
:104620006D631C1B0B81903F3AB13E98DC4CFB97AD
:104630009D494D99EE503649E2A396CAA61E5938B7
:1046400096AB20BA671893A4F850C6F7B2866F8766
:10465000A570A895C72732F33D53A82A4D0BED1F2F
:1046600036E2EE0025947D7341CE06CEB4CA384BB7
:1046700012FA386E9D40947164F96712F5B91CAF57
:1046800092B6CAF7D3DBDC3947B92DA98EC9D2035C
:104690008720BBEB933877C522F0A76AAB54C66975
:1046A0001D365E3114D168B59575CCCF2920B28CFA
:1046B0002F4F2C36091A088531251343C930FF0DB9
:1046C0005CBF485543C9210DBBB385454302D17A30
:1046D000904B2DBAE0EB259752C30A9791DB58C552
:1046E000DA24DFD7B3407C6AAF28E396FAE5663474
:1046F00070A85E3207F6C1191770CA15C5C1B8C5D2
:1047000060AF0A24A610AD1E554CA0DB57F318620B
:10471000E333B0230CE5DF5FC30B8D056CB3886119
:104720007D78C3450D8F937B4D4AAF01218AFE9D55
:10473000DF8456E884F7463C8F90955275CAB8607E
:10474000CE783E5389D974252CAB718058C52DF095
:1047500021AF2628AEA88E65D759B317664F1A56D3
:104760003C7242DA1EF3D07841CEA1C8719A1F057F
:10477000AC7DE6AF01174CBAF98F4781E2BBF78AEF
:1047800075E4EF526313325A37A9164FFBA716A2EE
:10479000EA0EDEE4CC39A100A7A659BC77C60A7E92
:1047A000F1B683184243710FB813D4CF8A59272723
:1047B000996E55BFC5C8273498E6340980D7A767D6
:1047C0006E0E41B53B8CD6FD94B5DE4DF99112824B
:1047D000655B03EC6213E9833CD560D2EDBC997E46
:1047E000E38414006EE3C9F143468B2179CBA29494
:1047F000B9B2B588725E06163F7286BB0B1A2F9946
:10480000E46C41089E18B88FBC52F108F8A299BE1A
:10481000A8FF143C32CF2BA099D1BF957C2CF6BFBA
:104820006A210A939441C2A279E9CA4EAF158BCD91
:10483000E4E5A4CAF070210BFD60CAEDBEE19BCC9B
:10484000D2DF3557822BEA217CA900FEC2081B3932
:1048500023B9D48F6FE7DF5F4F0B893C4387367BEB
:104860008736A009145753E296F84FF12891555115
:1048700036570FBD814FAF3BACB0D850673A26BA20
:104880006D9AB8337F4CF8F6C9FD9E4CD17564170C
:1048900091343C0A07DEEABE2606D56B022F480299
:1048A0009C66396501A483C49CBE9E7CC2CD2F1634
:1048B000237FCDFD62637CC8189627121E8A7B5326
:1048C000E586F5D701C258B65995E8DB864A6CF003
:1048D000584197276AD91C46B26C43411987577AC9
:1048E0001A2CD0AC6C1B33F4172A445FC2825B9441
:1048F000C86F3843D500B3E32B1E0CBDBD7C5754A5
:104900009E22C055DB5765BB3A1D18AA0BF5A51AA8
:10491000EAA4D5CDC79D53F8B22CE4CF2D25BA67B4
:10492000218EF6D50A1FFAF15844D5034E86BA6F88
:10493000131ABBADA36BF9B6E2369DD73ACBDFA411
:10494000B39E78F3C73822B181A224A4ABBE5B33F7
:1049500091EFE8A4EDE34F6C1AA773F656DBC4AAF7
:10496000AB35125258507476E6036CE52B7D6D5FC3
:10497000705619FC9FBBF0540EA3DA97CB85044AFE
:10498000FE8697C7D3533AAE11416DE13EC20A701D
:1049900019A20CECBEFE70D8AB8A37D5CDCFE3C3DD
:1049A000CECA27C507B19E8A084B155DF9B17CF0C8
:1049B00059A80C11BEE16EF38D16583F4AF16058AC
:1049C0001D0B79C883B7B59762C33160336C7857D4
:1049D0002F85FA12E587B34F779B07EFBA106B97D5
:1049E0000BE1B8EC3029DCDE1055A6E30C19738F0F
:1049F000A38E5FD1966D0746B148A2158CAB96ABDE
:104A000050CAF31C6545568582832B9FE287280C8C
:104A10007E61984017F35BF457E930A18B1E222E7C
:104A200019F506CA59797ABAD4F7FDE668F8E0E4D0
:104A30001935011822A5CB882573B1165FFD8B3A75
:104A400009A85D14400D15CA4FC69B3621D34C6290
:104A5000735417E6BDF3D3D58CCB5B468813F3DBD9
:104A600091D243C6CC6EF91DE6C68DFF7B27F88434
:104A7000F2ECF44FCFEF5F05069845598AE69D2288
:104A8000B3115271074C304364D8EAAA3C7661C036
:104A9000548EBD172BCC30B0B0C03A7E45B9C2D3CE
:104AA00062D2CD1619B55900515919586C9E11E3AF
:104AB00027DE6E8E3163C677BCA2CBC502F8F47FC9
:104AC000FBF49443C7C9C82EE13871A353A98E558E
:104AD0003FFE26ADBEFF8A11098BA07FA880F04C57
:104AE0007482FC6B429286CE811796EB34800377FA
:104AF0001EB4CBD4E8B27ECB14ED515C3822F0D892
:104B0000772C360C70959B86852B6F8CFEC8671DA5
:104B100061126D72E6DD282EF01C2F47A85D056F2F
:104B200038F524735105810EC73E47C44BA126C0FA
:104B300079F4DA0A83577A9F2A5338F84F771DD1D0
:104B40009BC8B4CB5A43F6E95D888E8FB82A3F7173
:104B50006AFDE99F8DDF1A8211017DACB0AFC10AF9
:104B600051EDED0A2637CA209E0EBD9830DE128622
:104B700003C160D8BA643C74FDD5CC81EE25F3BC8A
:104B800038278BA16B037551DE2BF94D42F69A6CD9
:104B9000EF2F332B18657B8489252F015E7FECEF87
:104BA00088CD3C60C3E752C8368F3655F883CEE2D5
:104BB000B5AC03F655E7FB7836CC75C5C62FA02CEF
:104BC0002DD170A5FDE5EAB83763ECADF74519D2F4
:104BD000BEBBC32BA27D83094F4B1F35E0C89BBFD3
:104BE00074EC48663A62CCCC5B44472F3C98FE1F7D
:104BF00003FF3C1C2C9272489A540D877B6949D65E
:104C0000845E302938138BD98664EFB1847C07AB7E
:104C1000812C733B37DE2A21F3CC0D46DE46F54E60
:104C20003FA62330673B45A03E49704C2B69535F3C
:104C3000A66C2116EE4E5030E1C0A8F7EF3E0F1FD4
:104C4000E626F9197DBCD0980AAA74EF5D28A6095A
:104C500013A87B9F47F55AC38798ED418252ABFC5E
:104C6000B104BCFCB123285D2D8FD02798AD48C37B
:104C7000E11E069B99A8CA4E96002F968CAA76250F
:104C8000F197EF652092C601762D388C5CA2D7D5BE
:104C900087722E8E7C16F662BEABF599A729F2CCF0
:104CA0005B14376656C7FAC3A47A83699321F2EC82
:104CB00052580D4B7C3BE9AB110ABDBBC4EC9210C2
:104CC000910168FA9C63D610ECCC59264F65E22717
:104CD0006445B03542A515A7E66B07B3F55CEC5902
:104CE0009CB874E50188278ED8C1AD0C00EA72B279
:104CF000B6712951C32A96A8A8BADDEFF1A689E0BA
:104D0000C2C28BD190E4EC46B9C2B5CB93F2BDCB15
:104D1000434FDCF1B00E29D6701F6F4F33B4D7016B
:104D2000745F398FC8478024E2D28627DFD994EC9C
:104D30008A28EE6D3C74FF2967059020AF8F54E5FB
:104D400054B3789245DD2A532FF3BF3152B8197E00
:104D500093BFA98AED23C23976BA9C2EC514B268D6
:104D6000FF0CD446C47D02BBC6564A875D76185DEB
:104D7000CACDF25FC240B0582EA404E33BB57D1DFE
:104D8000E409FFABC389EDEEB2244E6935A71CD907
:104D9000874D4B7AA4CB5F1A70FBB4B9CDFE730379
:104DA000114E572383B384694A9F9961FFFFEA5AE2
:104DB000470FE5DFD5E74C9DDE4586C13FFDAA7A6A
:104DC000A5123EB0612FFBA695DF87377A4591117A
:104DD00069CBE821A83F2FCA40B975DD4D44EF3AB1
:104DE0003A9842F0EC4D1B4D9996A95689D4E6A10C
:104DF000628694EAAB7F4101BA136CC668898B95D1
:104E00002B575BB9D62C63783173B966C103C1BF28
:104E10004222E46FE4990EC36E0E8F6490CF5D76EC
:104E2000B1976B547027E16B9D196762E8504FCEC4
:104E3000232FCFF5AF931E54B2FFA9BD49047C21A7
:104E4000B23723B3B296079073263F0847C6F48C57
:104E5000E4F15D182ED26B71ED30E78790F433AD3D
:104E600036373EE560B4874F8CBB210F01095116E0
:104E7000C366D6680AA44FA5ADDB05CD7B9B6EC289
:104E8000530A457C956A778DFF944A42B0A914462F
:104E9000D281F69A51A7FD118D6A86CF2FDB375F3D
:104EA0008D11DE7517833D2136424112342912E1FE
:104EB0004BC98904C18271F64A93B3C7656CAA3E97
:104EC0006543B12BF2D37B12FA329BB03F5083C6BD
:104ED00098C3573EA8D2FB0F32A5A4BE1037AF37F8
:104EE00079B0BE316D663AAFC70333EB4AD89EEF57
:104EF0006642037A513DFE10FA848323F7E3ECED1A
:104F00008982C4F23E6531D5749535CFBCB073BD8E
:104F1000CF43FD1C231AB3A24F4E9A21EE84AD83DA
:104F2000636606FE6EF50B03F88694A1C13915D8A9
:104F30007FB011A4AD0C83CADE3009316C54B712B6
:104F400069364B490A075AFE23DD3DFA3471EF7684
:104F5000A7038E60E70AA9B3F87BC938AA6B983318
:104F60005CE9291701DE755AACAA7F4689B7746CD3
:104F7000DB313904FFCE0A1A9845F083469127FFAA
:104F800004F11143CE5FED6BF62FBC3F6845AFB324
:104F9000A01226EA85FC7A1A31618252A09BE0F0C9
:104FA00077E2396F8245765C77BE7BCCBF1EB15904
:104FB000E2E30A005062C22A321490E06F6AC9A389
:104FC00032214C79AE69E8DBAB41A7A4109E7AC7C9
:104FD000029C7813C66E1D09F1A172FAFE3A0BBD50
:104FE000701BC9BF6221C9C9BCAD80F19F4B27E4CA
:104FF0001112E40DFAE0F04FAB215E1B1CBC815591
:105000004C692F58C421AE9041C552A7C41C6AE513
:10501000A78B5E29F6280CF3206F1150A12F864430
:105020003B210A3807B16EDE6F0EC3D6CF1454177A
:105030009732D641866B2B73FC360106A5C09FDBE9
:10504000307144E2067178B706539F150393CCABD9
:105050007B536C617B6E97B725CADC9D2DDAA8A2C5
:10506000E44A88AF102376F50108FEB781D5D5B1A3
:10507000A98BC86BED458895DDA363D6C778036817
:105080002E45682F3A50619F70E8BA23A761738854
:10509000BA4F6B677D71328EC0D87BFA337352A7DB
:1050A0009A7C8601FE5D16BE07EF4F3AACB9AD7A29
:1050B000292588C185E08D94EF24621FBA900DF5F3
:1050C000E74908A52C00782747BBB219D42874C932
:1050D0000BC0AD0F446F8BE1AB99111FB2F3E06DC4
:1050E000CC03BB8C9E83DD42E5ED4DAEE378C4740A
:1050F000D009D1C756B7843C8BE38042F8F6881FAD
:10510000A0A3BBF7107E191F4F40756D3CE30D60E7
:10511000D6AF405AB294241E78ABBA3177190050FA
:105120009A63401EE044EF60B0B3FCEA6D3D2AB0E4
:1051300044BBB0126BD47F95F5AAF0460AE57773AD
:10514000931BC50990839DF6F3B445E6B82C1A333A
:10515000836A818AD5EBEE0958FAB7ABDA7D9BC535
:1051600030D2E02C1DA40EF07218EF21C8773C223B
:10517000798D5CED5FE52861D1D4BA181E818F6A04
:10518000B91CDBA87BFFAB6F89622DC5B6F0FC4C68
:105190007E27B396492AF2DD8DB8FBCC6FDBD69023
:1051A00025A42A08DD3D8094896D073E0821D7F5A6
:1051B000C280FBFC2393068371074B01B63D022E90
:1051C0000F2A4131B1DDC33FB805C8088B2706B5AA
:1051D000DFDD75AD7BEFA008C210D8D1D78B54FAB4
:1051E000DA9083B3B36EF946CA7FB16F0B351A6D8F
:1051F000F7435FCD5E6F9156C59C10BF71E02BD415
:105200001C2644D524AB4C198732806FB3CEA64CF4
:105210000F6A82FD504D7D3ABF8A9B28F35C73492B
:105220004BD2E646F44F239BE7B12A96C3339196BF
:10523000B46F673706E618E8511BAC47551AB983B7
:10524000C5F3ED76FE37BEA59610F3E132386B9CC0
:10525000B6737EA7A2AD094F78C0D7EDF5B043A7CE
:1052600037D7FAA488DEBD2A8D0271165474D53F53
:10527000AF9B5922887B0F6E642E6EDF165548E374
:1052800018713D5AF1E496D1C68C9DE42AC9D72EF7
:105290008CC5664600E621201F078FADF2F8F4F5B5
:1052A0006C0245F10595EFA821352F479127A19C68
:1052B0002176163D85A99D2700583217793D8974BE
:1052C000B2FC5248751BA5B3E0F0C9C72BD7B7276E
:1052D000C7A546F0E4AB4B31DE21A61A662D547CFF
:1052E00056078A38C7F965383EB25C46725337CDE7
:1052F000764D8DD31D5F404F947403A5BB3A56572E
:105300006528AF065A8CEFB09E2DAFF57AD66C6942
:10531000E18D77DDE507F84FE294B59B29A704FFFF
:105320003811281AA749008BDBADD05765A3293E59
:10533000F69C94DFF89128B9E9B71621A16AA6ADC9
:105340009148724149DDEB3B39A916F15ACC042D45
:105350003BE167514976556755AFED9F2F7291F646
:10536000944405434A7D3D635EEF3F854D1AF961E4
:105370002BC14663CC421651ACAD9DFDC38903AC35
:10538000928929BCE6552733D8A3022A44798DD6C1
:10539000417826C356CA112DCE2C79461771146A4E
:1053A000013232C4410981D32F84F0F4EEEEE8D704
:1053B000A0B4CEB07B4368C8C725A19B1D50DE6951
:1053C00047F0FDA2BF15D3F2B552D1CAB8EBE1EB5D
:1053D000E9821D06A7EC5A82B0723D0254467E9EB9
:1053E000FAED95BBCF11BE1C9AF7A7ACB71671E4C6
:1053F000AEFA4B0F253876D7701AAFA1019BFE236A
:10540000D60BE8D9B5A6461D1DFBAB1A183B0ECE30
:105410008947FB4C9BCC2D675B0372A4A0F43859E1
:10542000F74A9101F487995A6AABD36FF483B59D1B
:1054300003B135319A721A5445CD1081D290F5F7E7
:10544000DF605B8D939D4933C97E76EB8C543E8B38
:105450003F47A2ADFC14734D1DE42BC14F3766BD11
:105460001FEAA84D8CED922A410C0BC5996E81AEB6
:105470006F42BB79F4C2C1CB0F8F76DBE66F1D9113
:105480002AA97AAB32EA57C59AE6720CD4C171FEEA
:10549000651DCDB7971AEBC44E275935A4AAC08312
:1054A000E14D9DC902110E6C4C4B71F0ACA91F92DD
:1054B000250BF4B39B278ADF350017A1A9C6ADC61B
:1054C0005CAA1FCD14A47457F36D9CDF8E3134B0E9
:1054D000049BB68D1F8DD906BD39A5965CDD238949
:1054E00014525B839C63D67347825CC31C18C78AC3
:1054F000E8A56789AF24AF85CB3A8F47D7A8587105
:1055000093776B02CCB6A1641A5974F79340F0C933
:1055100029AA5C15C8C5E4893DB6E9C6033D6F32CA
:10552000A2030F68F637379416D843D050C1DD6D0B
:105530004F14FBF22646E3989E07B66B8E83F4C4A5
:10554000894861A744FF6BE4F53F08EAAE4CBE2CE6
:105550006B3B9D1C51C5C97EE8C12AEEEFA61874AD
:10556000BC726DCD2F03270D3B46C9B699A987A9FB
:105570006CC010E617ED71FA61521DBDCAC1E1E0C1
:105580005B7BEF19E10465A09EAF9E5E99D5FB564B
:105590009A7F4426C60D24536CA22CBC1A3194A3C6
:1055A000039FCD5AFFAB082478E9161627488F11C0
:1055B00089253A45F243CFD5E4BA48CFD35D630C91
:1055C000E16B0BA0E1369ACC6FA82FD3CEA8EA9955
:1055D0003DEEFAACC4A6760AC9B3A2B4233A556329
:1055E0003F5500496AC99C0E0D949744209A27B2F2
:1055F000C5858350F098ADE0F04DEE7CBED323C35B
:10560000BF0105B4B6767BDCE771EC536ECA5F353B
:105610006BE991CDB330F44FDC55B77EFF8450F881
:10562000DC5B99FD0E858891F8A57E5F55973D1747
:10563000A8EDA106366736AFEDAD81326B7290F002
:105640009D32DC7093EEFA679AA3AB699DAF0CD4E0
:10565000DFB0F9D2B248EB6AA207309476E824A30F
:1056600011BFB9C6911EAFCF86992B966C0297DEFB
:10567000CE183F0152B209FE3ACFD25670153DE620
:10568000B3CA9B1BCF44E69FA46E6EB98EC29689A7
:105690003C6A7CF800C387E84A9956B9E3BDF6C76F
:1056A0003134923B33ECE35356D071630B73E91002
:1056B00088CAFCCB8FE84DB676D97D0F7FCBC4DA94
:1056C000991C3137487CA72110A7C94E67D524B94A
:1056D00034F5D9E3A4C6307A80B2CCAF25C8FB8DAF
:1056E000F986E64B2AB16FB7761BAB115BE58EE905
:1056F000382C02F5BF43230A7A9F057310CC341669
:10570000CEEEDE55AE877D975E3552D8042AEFBEC9
:10571000EC3385A147E9562071EFE8384595148DA3
:10572000F757D38F6087E2F69FF0543AEC7D92FBF7
:10573000EEBF9BF2AD451D3FCED79CCCED1C39335F
:10574000A5D2851D5E0837C912C0EE8778E135D233
:105750006F0B423B8FEE888CAC72BADBFE17688A07
:10576000EB2C3D911DC9777144DEC3D4DC35ABE130
:10577000CBE9824898877962A74F6D4C7BC051B3C3
:1057800092A64E7515810ACE6B333FDA63599E9708
:10579000D3EA21D95E211E8D2D1A444956C00BF340
:1057A00051C6F7C221AFFBDCB274995E8C94660CD3
:1057B000179E03B4714A63F26501F7CCED19347496
:1057C000560A5B81AD89DDCC458DD8AC60C925B565
:1057D0007FE7545A2A1F0B5D05EA1FC25B4E3E103D
:1057E0002B325E05560B724D13E5257516C075A15B
:1057F0004FF476CDD63B833891079A5612E6BD51C9
:10580000F9E67DE75167ED2B6DFFFA5AE72118E6BF
:10581000E8F9E41ABFBF3B79A1F74FD29D69B638CA
:10582000456FEA2A0FCDB461599C1D9CC8DD7B668B
:105830009F24E310DEF79B261E3A5F8A8BF798C8F9
:1058400006ECBC242A337C0C9D264B4C9E58B3E1BD
:1058500059D756C05BDD181FEBA109FC86314CED12
:10586000A94029C0AE9C6A04D3BE1FCB5DF9D58484
:105870001ADE89F317FDC719EF54D45260DB571EA7
:105880002E6C08001B21A44B36218B5C4180549365
:10589000D95A2B67A22E0A02956F27D5F6BAD138AE
:1058A000DE44FF1BBBDDF7EE2736E50CDFC18DE8DC
:1058B000B3523BDF83D3C669D3B9EE8ADCC2238EF1
:1058C000180D83B39210B2E10A24DF0EAECEFD862E
:1058D0007EBDE670761B7E817D59497A59DBD528DD
:1058E000435CB19BB4FEBDED38985FD643918D4DBE
:1058F000008C78918AD86F99B6A5E8E0B09EA90689
:105900003C695218D15392728639FC0233B204E8D2
:1059100063B159BDDE9198E5AAB29B1259F70AE826
:10592000A01E3B20310390B6B81B5C1C9CB2697D65
:10593000148C883831E4F19C494D5534587F95E1F9
:10594000A62A096F81376E3B32AFAB651D11A6FCED
:10595000BEAE4B07CFB4EE2DEE057CF82BEF09EF72
:10596000B309A95CF2135D9A561A9A23B0870026F0
:10597000EAABC026E404B90B694B659F0345C472CA
:10598000C80B8645227E3939EE2591A6D16D634438
:1059900012D0D2D048BC5E597EABB65F775F3B6316
:1059A000C738FDC86089F7A4E2D7810C75655953E3
:1059B00051B11BE5CF70026EA9006938DDB5E5A3D2
:1059C0004E705BC332F6D41BFEDA732790396F0E2C
:1059D000056EB98B1F3EA11EA675743FEE8AE4C00A
:1059E000039143D660091BBD8747346C08463A30A3
:1059F000B83338303E16652687012AAFA68D3D950F
:105A000096354EC31650E9CFCEEBCAA28342D20BD5
:105A10009C0ECF942707EC334F8E12D98CCB3AF1E2
:105A2000132C4ED13095DF62E398A6A894064F5B05
:105A3000CE3ECA61238E0C47D8BDBBBF7CBC773637
:105A40007E22D5BF78423A04B2668F1910659671EE
:105A5000C54A56DBF78BAC645502257D86D8A1D8A4
:105A600011B24ED136D34044EAAAE889E45111304C
:105A7000013CFD2BD50E33A3A104663554CBBE6685
:105A8000B6DCD1F5890EB167A322C7E533CE406CF1
:105A9000778FDCED5F81CB05FB9B2DE8BB25CD7DB2
:105AA00012FE7D0BCC389F42CE234D6B3B920AD920
:105AB000E4220B4F6858E9385D6C39AE8B4A149E6E
:105AC000181CA86F841520FF540DA171ED1F008ACA
:105AD000B42F9C38BC848BCFE972B1366F8A56FDE7
:105AE000E065E97528EB6AE3DFE2A91640361DD1CF
:105AF000FADFFE28CBB5FC4113BE1112F754EC01BE
:105B0000E4C366947C21FD0B4223458C2AC30240EA
:105B1000EEA4EFFE5D819A3864F7FE851E7305B42E
:105B2000EDD3FB61C992DE5F2F777C03E14986E309
:105B3000BF8D5C45DEA01D8355759680E6DBF606BD
:105B400003B4EC22B3AF7F3EE03402A2ACB75B32C9
:105B500028291AAD27D3D4AA9223672F5EC85702EB
:105B6000AF13A00E3A1E5A9879C882BD63AC6F84F9
:105B7000196CF5F6C800AB51CE2C7E8EE8DE2B42B8
:105B80007E7C2FA8A9ABD887883812F0B3EEC52940
:105B9000E94F25108E627B928BAD051EFAFA69776C
:105BA00049D978F66AE8E7DA05F6970C09D897E557
:105BB00010FE47F5F1DCAE1F0E4FBA5C14CB87BC6C
:105BC00084710AE609049062B8BDE970DDD42A4AFE
:105BD000B20F4B3E298F4F60865B46D8002ACA140D
:105BE000EF012BFA243509B6D900CB8DBF5CF594B3
:105BF000C5FA37EC5D80A28B088780A096037D7183
:105C0000663DE8E4FB42D93A1B18C152664EAF68C4
:105C100006CBFC0E97EC735868A2BB94587B368B6E
:105C2000BB54CECE77EF87CC56C17F12C3C6E29F5E
:105C3000FB5F054580A2F3E01E869D9167ACC6D54B
:105C4000CA93B7393834B2085246C962C19629C6D8
:105C5000E3FCCF67C2BD52AB7F01E28673B126BBC6
:105C6000A895C76BC6CCFDD1C56FBA49AB4E67804E
:105C70003A92260044D1A3584448CF406B138F6614
:105C80003FD28B6CF81A926B2BAF4FA56C38694FD3
:105C900099637462EC1088FAB98220AB20C16D045C
:105CA000172D86C68164158CCB84D8103813170C39
:105CB0004B7ADE9B630B598C247053017FD54A6964
:105CC000C74B08E3271CF88CCAA49136A45EF813CE
:105CD0008D47B2EB6C6FB1E5F8B212CCC50E430440
:105CE000A5FEB000FBF0C6357C654E0D18F1B59AE7
:105CF000B93D8891CF936F5D84B5823EC1BB43832C
:105D0000B3DB2B791479E66058DBB66A9AA88D6408
:105D1000D2BDBC7A1B489BDA9397454F80A580E69D
:105D2000BB2C72B7E0F2D7C094ECEEDCEFD2260BBE
:105D3000CC6193C19A9C4C962A0EE5474D63DE6573
:105D400092A07E77CC3E20F189FBA8740D9B8867DA
:105D500053FE3DB282280D0DA9DF389FB1EE3B6A9C
:105D6000BB49AEF32E4E7B8394A706D2CD54E927D0
:105D70009D66E86DDBAB4480E94A16E61B827843FA
:105D800017CE50163B55A1C2A70018EE956292BCE3
:105D90002EED7D97A270FF023C4766FB4388AC90D6
:105DA000210DAD38234C4296A483CE8EB2B99CDC33
:105DB000CD5B20D721CB56CEBA3B8747FCA8ADEAB6
:105DC000A2A5EC0E917349E6A280F642C08560DB85
:105DD000B844FF7E20366869A004F75D4E14544B2A
:105DE0008C2D868261DE767F75CE8A3F9B52724310
:105DF00006A4AA181F83D4EBAA24D6BCABA58CA9F1
:105E000017C93DB3A3F7D9351ACFAB2C45F7E2E755
:105E10009361950D19D7A0362F2CA2B7D103FD435E
:105E20008BAEEA293A5B0E02541EFC1A737C56D0E4
:105E300040F69AAF851E19C13A27B3C73FD46223F3
:105E40000A277E7E00CBD7E1A383B34C9A15D46E8C
:105E5000DDAA08949756944456078966B4F6D3266B
:105E6000DD086D3D55E1E280794D98D5A074184369
:105E7000DF334C9E4BFE1481822632109B8B081E12
:105E80003F0932D32693C180877B9A8F300385C127
:105E90008223FCCBBEE67637328CCE461498992B03
:105EA000DC8D6AD20C432B388FE5B1A5A63A8F2141
:105EB000888793A1EC538025A57635D8468925554A
:105EC0000F194E1A99A3889973E1DCAD6086920B85
:105ED000CF1E65EAC4D725D3590DFE4E20535C3B37
:105EE000BB44B178975D25BE6CD614EC710D4B1494
:105EF0006D2E9C214BAA954BD3689361B7EFD99433
:105F0000B076AB6A1F642F39F9AE9CBE507EC25387
:105F1000700BB00A9301137DE1F11087328C6D1282
:105F2000D9253CF0C32DA193D200B297FCE3A17117
:105F300063A3D3B083881E03B23FD4CBC48A2E445C
:105F4000474A903D47B3BD584F09C9085BDBB4A52C
:105F500079CE590F8C3D8B94FE093ECF745B402D5A
:105F6000C76167A0610C7B0F6ED131483EC0075DF1
:105F7000A460898346224541667F80C12D91935359
:105F8000F23F1208CE441D849F26ED8E767440D3D6
:105F90002C28BA6234A9D060EFC485B4912DFC35A9
:105FA000E4591D29A3CE00687D257CA18CC9A88A4F
:105FB000ABA1B0CE76290E060D48219C7A5CD3EFBA
:105FC000BC68EC267BABE56252539E83F566175D99
:105FD000A7A70FFBFDB7C11E9190F16CEE9D6BAFB3
:105FE000114CEB68825E9BF35D784C710D5A1D6D10
:105FF000061A79E118A9B045C6D754F6F68690BFBF
:10600000C9DE04E1DE8F13667D3E8C3378725C8DD1
:106010006F01C5BCF2B3AA82DD6F43A1E9A0E2FF24
:10602000ABC760BF48CBC0724BB54542B2D566E83E
:10603000E59BF65E0E84C44B446760FC718A693749
:10604000EDE4EE48069BE9BAC95E10218720176D82
:106050002BAB885572B01F04539937C0EB2D050444
:1060600033062CBF6BF5C895B132D7DA578E524440
:106070004C89A356595F24BC04B33958C65281AA2F
:10608000D470A3F4140F2E919D93E0A1CC89C1C2CA
:106090008A816FF7F49A281D73B28F09724C6926B2
:1060A0002894CF795F929B20D0E1B87E11672ACBEC
:1060B00077705D7C255517054F1D57A700D88D13A8
:1060C0004D963E15806CE6B2EFC89D48C96EDA4E1B
:1060D000D88F509F8DB51D2ADCC6202BF9F199F77A
:1060E0000ED5F213DEE5B886113CE226FF02CE6142
:1060F0001DFF7F33108340F66F916B92259BE79BCA
:1061000023CA5744F983EB9EF2E1DF222B87052A4D
:1061100050BB86F5299094C9321B57DC2E2E8881FE
:10612000CC69046731F0962AAB95FE1C675A8480CF
:10613000F91C59CC11E677C29A4281A5E9D21D0615
:10614000F71ED787395C08CA4F572620C8C3A40D4D
:10615000CDF19F8E40EF92E29A494F889D7D19F3D1
:10616000A0F8BE9ABE5482E9A6CA026482CC149EEC
:1061700047F028A8A1207CA8760BC6DAFFCF351BF4
:106180003B704A76852F2F7B373EE66C69AF48829D
:106190001EE3DBB8067CD26E0DDB45009F6736B38D
:1061A000897725D518A741DAA25319813309ADE9BA
:1061B0007AB5CDF06D5AF6620E8ED38B06219575A9
:1061C0001E3A947EFAE6F64D91470FFCFED077EF2B
:1061D000622261AC63636FE20E622182EEF113AF63
:1061E0007836ADA07B419D796D9C0D2A312380B01E
:1061F0002B1AE9CEE0E30902AAD06ABACE7BA960E5
:10620000964D8CD02D1D220DCF3599C1173B766050
:10621000119CA530FB583102758BD4CB462CF5EC84
:10622000BD6CB2828B6A5926FD023D222F847649CD
:106230008DAC6407428E08C8CB69892B34014D327E
:10624000D3820A620C9D2138FA52E6EAB0B855BCF6
:10625000D901A087607155C63A0E45F4B442212297
:1062600038E0573C44C3D6FECF18165E466C01B5E5
:106270009993F63A617CC1AC29241F92BB3F1D6CF7
:10628000926ECCE26C70D9F12C9AE909E5CEFB0351
:106290008153BDEF78803240A3D75A7787C7B8E6DD
:1062A000F6EAB102CB8A42ADE4B50C20EA8EC8B75B
:1062B000AE422DBFE453615C0FACEEBDF2186E0927
:1062C000967F02B2B10B40E11D2621B6994C2B25D9
:1062D0001818E888D384A1618ADE376A410109C1B0
:1062E000EB65E0862ACEDB2DAEE5564F8BC0A5A927
:1062F000B9EA3F2E1D152A18F6C09294AAD0C459A7
:1063000075BA8F15E54EF99C052714D3BF03C9C292
:106310007F826541B7BB87BD67BD6B29668675A760
:10632000AC28EB194813D4EE2ED1DEC30D5C0F0060
:1063300053B0E47B97EAB1BC7B3621AACFEFE4905F
:10634000B54E959FB534FE5C58A0A7477E747C225D
:10635000D7EED09C0321CFA11A1153985222B30833
:106360000C28CBC3912AE7B495EFD12E28337B9E1E
:1063700069C59A9BF9B7DF1AFF0D254B7997A51DC3
:10638000AA9B2A94DAF3DBFE841BBB1AB32076EEB9
:10639000CBB5D83D34B1F69E88F3AC4642377CC6C7
:1063A0000620BFAC2F31FA942A24387CBE84B50273
:1063B0004EED9ACFEDB0D7EC24A20956E84950C76C
:1063C0000FF168D4CDC4A16B00ED0115980419FE3E
:1063D000966CA4FBF7BE2983DF2999FB0D02951D5E
:1063E000FAFC4C4DD110E28C5D7BE78EF55CD54C10
:1063F000FDBEBB51DBCBD97A79B27E5D83D3759775
:10640000099A27AFCD39F6BEF184D6964D9F532F0A
:10641000A9576CC5B0E1FBB9A8BE5DF163035FFA93
:10642000E9885C3CA9BED3E6C4ABB184DE1330007E
:106430003014CB2493595D6442A65AED9C148FF11D
:10644000A91904A0611BCB602B0B31CF4EF08D6AD4
:1064500026B80FE4182AC0D1A0B0D1950A09940833
:10646000E3BAF882663B8B675B0D5242B89EF583B8
:106470009999A335CA12326895133A15F71EBCD103
:10648000459FABDA4FC6CA1C62B69423BE24B6340D
:10649000FE8484302EFD27052FC0C7ADB193CCBB41
:1064A000C7C3A46C88FF419C5BC323B0F3D6C9D497
:1064B000110BC6C5392D7888BAE8F7368DF9CB06A9
:1064C00070EFF033194738049B9D3A4E0E31A47596
:1064D000F0C5E0433310601F35F7FF76931C9ADA5E
:1064E000874DB5B27FD71A93A19AB4159B9D053EEF
:1064F000EAB62B2F5A43E99F5224016FACCEBB3F23
:10650000FE1A54BFEA0C755FC7ED79501F04FFB83F
:10651000FE974790DC1E8B5858BD4805FB06137943
:10652000DC6C60FB7BAC1622CB30F8A217E02DDBD5
:10653000CF70388FD5510F133E480840A1F879A687
:10654000C19DDC3F0B8E54F14FB08AC300D3165A65
:10655000CB87151D7A02B8DFFFD78502FD5CDBEA29
:10656000EBAAB4EB78C572169E595153A07BC32396
:106570001BE482F6E4AEA93832B6718018EA6CE406
:106580003D639132171DA2B20BC74680685648542E
:10659000182D435739E6B5224257784B82C33D2226
:1065A000D0B18EE9F0A72C756C9F920DD5333621B2
:1065B000E30C06A647BB8A626C00F1648FF370108F
:1065C0002157A6F2C7D7BC5D5EFAD145CB39C75477
:1065D000922C5B8CB711D721753D57BD1C57DBCD75
:1065E000B0BDCA688BCE5C90B978D68BC5ED999456
:1065F000149C854505F4FF93FE4DE163C4CF8DA146
:10660000FBF3BA51C4B4192D3CF908907AE9A2E021
:106610008D3EE8B0B8561683CDBC477867D13E0AA8
:10662000D715291858C646A0E0676C839057DA9DA5
:106630008AC1337009829132FD8AE7232D9E791237
:10664000240B747CD1BAC798D12FEFD876DE6DFDBC
:10665000B32D1F1A00922229203AF874E3D7609ACA
:106660002C70ABC56786D3EE24D42FF9B811831CE8
:10667000E6C055EB82836FE64C5A35D570F7FFECD8
:10668000899F6055C65A26D7BB81B9092C6CAB7F50
:1066900002758D0F4580E667D9DBF0EC208C2192E6
:1066A0000B0D281F58F00CE47EAC459DAED0A6D74C
:1066B0002D6F7F6B21A5DA7B4F6C132414924B0155
:1066C000F30385B952B238A7E92EA0BD56529A57A6
:1066D000679275664F268B1D49FB8511BE1435D513
:1066E00085331389E75BE8CCC9ACD9E93A4FD810B8
:1066F000D91913DB129198823AD17FDEA9C23046B4
:1067000097401B347F2C14C7B6B34D345390DA0036
:106710000E97A8646DBDFFC6329EB4C126D24EC886
:1067200012FCDECBEDB7455B78D60933347E95AFEE
:106730009259139AB620B5CC74ED5BD82CE7DAD415
:10674000DECEAE11DFCD61C17016EC6199E75CC29F
:106750004BF2461DAA75BB33CA5C20C81923029CA4
:1067600068F684DCD3D12C7F0FEC829F2E79245ED7
:106770002269378F3258C46DA9F06B8DB48B5F904E
:10678000DAC7D74A146999CE6BB1967DEA27DB1335
:10679000602B7E5482119EF6F0BAC4A434B9B0B511
:1067A0005B33DCE4E3261BD1C339375B845873B118
:1067B00070B9A10E62087FCA83B36292F9B24869C8
:1067C00094F3D25E2A5886B7E9BB8736F056B33FBA
:1067D00085EE939427D54AC1E33B7DA1601915ACA2
:1067E00003BB32D1F26AFC8942E217EE343AF7A8D1
:1067F00042C795F23730AD95B4C0FC56BC28296F1E
:10680000FED6BAAEB748306C480627FC39B86F914F
:1068100067957FA28BE63A9F9E6BB719E791B20905
:10682000F5ECF06E4C96A4EFDDF8703EA31A1C5107
:1068300011D9411642F11BEF7E3A3F4D0431735599
:10684000B9FBCCD098DA1042ECE4E9729726F15308
:1068500067264B61D2AF2909141D1F69FBB5E6D02D
:10686000FFD33992AF8B0CB0DB22B32FD69B0D0731
:10687000E9F68AF528ED4AA0A8137C5B9F736AF7B6
:10688000DC37FBBACA45E6ADD678E821D1CE67A29F
:106890000E8EE7F042DECC070245FBB13D191A9897
:1068A00056E907914496DDF9BB0F8EF3F12EE652BF
:1068B0009A5912D9253F0DA0D8FF4ED644D62DC9DE
:1068C000D461E9366D786AC50CBCE9FBD9FEBECA55
:1068D000136748E24F173D3E0F24C640DDEA6E388D
:1068E0002C9D9648FC479438336F6FF5C4A05381B4
:1068F00073047914A4C156DD06A558952A2B6DACF6
:1069000080517509907FA791D35F22E2A96C4B2833
:10691000350E8A48CF7EA79F5456B954553846CC79
:106920002C7B4E3AF1B50F3A2D64897AD4F2108E51
:10693000C3250FD5D1B3140FFDABEC2ED49FD07E61
:106940003D2B9851FF6737F166D9C1D39172299ECB
:10695000280E1BE00634BE788203CD8E6BEEB19319
:10696000EE88A9D734A5F5F173D02446D7BA56D905
:10697000766FDD78E6611006625C84E6AD405926EC
:10698000C9D4ECB6A8DE1B85EAEA6B64591FA47073
:10699000DB450B4341F89748D4D199C5D4514034D5
:1069A000277C2CBE046EAA44FFD103D9E9D728085E
:1069B0000C27CE89E2EC42F283C589EC230472B144
:1069C00014FEC22E9A038BFEA6B361FD3C4342BE69
:1069D000E679108F3CFA639BF590E2905AF2832E91
:1069E000D8F61FE5D888A55BD71F88B66965706F94
:1069F000B9B7319D37F28E7807A28B7E6EC9C55725
:106A000047A410DA78BA69D016CC2EB72EAA4C85D6
:106A1000F608A972EB3B97F788C02B438AC3ED4178
:106A2000A205D6513AA0D79148E772E1D2BF4CE710
:106A3000AEC8CA35CFBC45DCE9473CA0CB68003FB7
:106A4000B45E3828A3E653EF207CE3B0A8064A5E84
:106A50008C51179CF9F6B77C47F18A4D898EEE511F
:106A6000F8C4474B64A5BE6EFA6012BCFC611E07F9
:106A70001816A94A1884D397C22BDBE348ADDA3C39
:106A8000A447D9E781F7DFA1DA3C23E49037E24B52
:106A9000E4D5808001FBC143298C23AA8BCFE9C1B7
:106AA00052125274BAA09825DCF647760B2632C5EE
:106AB00072C5A5872FBDF5479AEFA9190E9BD7611F
:106AC000029AB99EDB54955FF43596F2207D416AB7
:106AD0003472C75F483D18DFC9BCB438D9D9D1DD9D
:106AE00094A083C7C01A452957D0EA008008D71B55
:106AF000C9EADF0698A0B6D60D3A1082C2DD4AC0B8
:106B0000D8359934F3026D8D93E34A63766F5CB0A8
:106B1000E59840694A22E348E2CBEF408F8FD77077
:106B200068D3476BB03DF2C3E33F3006A9B9F1EB40
:106B30007F7E215DC59990A74ADA051F2D98BD4833
:106B4000BAFFA8E1C635552ED041718977CAF9E35D
:106B50008F5AF8DF73FC19651A9BEB7737D772975A
:106B6000D244200D5D4CD886AA1A66F0F2BFFCFD17
:106B700076887B5F26CB4F5106C8F7CA243873F05E
:106B8000FBE7FD0AADE9C5F5FD5DDAFCB0E0FDB05F
:106B9000DABDDF7D4380D14E3479C9E5673A067BA3
:106BA0001A85B323096903BC96D78AF299C8589409
:106BB000315EB8137C328D87AFCA56629191F0DC9A
:106BC00069B4953858722B1FD1BF11F8CDAB2E1B6D
:106BD0007B27C642E84E6EEA96D1EBCD3B0D1C1FDB
:106BE00033CF0C84395D28811E9BA4B64012D4C4D7
:106BF000F4B512DEA4E2B942FE4CAB585B177660E6
:106C00002379EECDD68008756D51AAE2C86551C8CA
:106C1000FEE8BFCCE215A25982E4986F89E55EF6E2
:106C20007EDF5E564EA20AA154D86D4FA8F01A2FEF
:106C3000155E5C759673298A7CCA69433854890746
:106C4000C2AE838D2594305A748D3BE28190E38DE2
:106C5000E1417646D11E785CA67E79DBA6659C284C
:106C6000D8440A4C3A400D5E237AF8F81556AFED39
:106C7000F200FFCCDDEC6161727FD7317B3109F02E
:106C80000AC5F6C8412EBD2268A51CF43DB1F32FFC
:106C90002EBD05C26AE19C595FE8A99CBBD49FD177
:106CA000E983E38C27623E72CBACD4B5BE7E60B381
:106CB000248771CC1357D40DC315DD7F76560EE1B2
:106CC000E0AA62D0AF989FCDCE888C94EC14027469
:106CD000B918391B2C6723D7D0EA123CF05F5E2429
:106CE000614BFFB45748519E187EBA107E77B0F0C2
:106CF000B38C6D16DADDFF03DDD05E5E91EA78D7E6
:106D00000752A35F2BDA30632E9BA1D476C63CE3F7
:106D1000EBD8B4DA66402D51D9EC18F0B8B41B307A
:106D20008D127B19C0FB809570EB24B7E27839C8CF
:106D3000EB5113F067638821F033F8558E41CB5F38
:106D400097A670AA2AC02D7EB738D97E057923A4CC
:106D50001A999F1A2E9469106E5FF09EC22D39C247
:106D60006F21CAA44B3EDF09D84B84CBF7196E02C2
:106D700085BBCFE5FA6E06226392687C7C52D5F221
:106D800020D948CF9D65BCD567B7284AEFC0AB4E28
:106D9000DC4887388B35B419DAA2B92F48004B2666
:106DA00012011BB41FF55956A2E5CA25CEB47FF5D2
:106DB00081E003CA062761B4C0B9AF1E9D1B68AF4E
:106DC00038CFBFE131A627FB9520278B4B6050EAD7
:106DD000909C8B3D76E9791AB796538C8B29E9857F
:106DE0001279D5CB2E8181C922C4055B6423581644
:106DF000BFF92FA89160609D6C8C6E80FA68444B3F
:106E00003DD13978F7E014F0BDD363749A4BD5F5D2
:106E1000119CB4F3C12FD3ABAFDB177B7376D9C50D
:106E2000B1B5F0F48CF88E40DA590F4AF5AC66EC47
:106E300046B267F66D30CF5134B4DC114DD3C15436
:106E4000448CD2B31094CDC369AD88CF24AA5A62C2
:106E5000CCBCDD48C0B34288FCAF3A729B20B97706
:106E6000A2521D5965661E145FF366C024074FF2D7
:106E7000C615D0DF48B0E4F1CD3891E408790CCFE5
:106E8000511C9642CA8F4D970536E1C31398A7143B
:106E9000CE6D7AA026A1D7922DFABF2FA40A442D39
:106EA0004F10186BBB0D39BB6C6BC179AF70368856
:106EB00029723E5049D312E4D7B370C3EBAB959718
:106EC000147B94F8F3D00B0F1C4E9ED8D8AD662DD2
:106ED0003C7F2AA2BF948B07A804747D9D6EB815D1
:106EE00064219C7E6C27CB181624B8C7776F114E8F
:106EF000AFA589D6E7DB6A538560897252FDC50567
:106F0000AB879EC93FB56B74730435AF906005586D
:106F10005448BCC14669142874CEDC794C41E9D888
:106F2000CB82FE67E774F1BACCD53B4FD5E9E07967
:106F300043F860160B4CB5440A6DE663B2D8F2759F
:106F400058C8FCBEA835860078F41CFB6D4A5A442C
:106F500035D43B9C924E146B088B7695AA27B4D6F9
:106F60007E93EB1CDDC4CADCB2DCFDF8862619A1D9
:106F700010164678594086B30324AEE97B1C572E81
:106F80007048913A041ECB32C424F1E1890E2B578C
:106F90006CDA99A5827E3354DE582FC0DA1B02EFDB
:106FA000D3CDE7B25E12F4C84EBD6A41773CF90416
:106FB00030C0A157525BD24C609755EE3D6519CD5C
:106FC0003606E4DE38F3022D859659A295D81CC802
:106FD00005EDCE1DB94C31C1D1CA36E62D66A5D11D
:106FE0007B13F5F38E5CBCB7979E23F79EA897980A
:106FF000CF04DDD0F717A09883C7AAD25D42190944
:107000008E6AC1E5BC0A41C0D0EE39C374BDF11827
:107010001B6AC4599320FB757C6D476BB010B28D11
:10702000BCBCFAAF2FD40FFEB0455C0F41696E6057
:1070300062D891FCD8FD42AA198E31198E0DBF621B
:107040001A620418700D77452F69DFA1DF9DB4A681
:10705000D36C8CA69D38849B26B22802957F82DA59
:107060006777C1B706767112DB8EB2899D86FDDB2C
:107070009874D59F3318AE7EE95E67224535A06EC1
:10708000050AD0856BA1C6BAD0404A6907A0DA9B31
:107090000CB46E3D415B85C4B045BE1CA5DC83E0ED
:1070A000A9284FF9550A3E44E177AF4FEEFC066838
:1070B000070A624A628C975721EFB06C7E0794A34F
:1070C00026E86D4A19500CC84534EB2869308D11FB
:1070D0005349911928E7924A961C515A7F32589E7B
:1070E00059BAE5DBFC8A2C87A929B0304C3747B167
:1070F0002AB4D1E965C87610DA6407AEE15640508B
:1071000073F63DB97D0597332F1DBE6FF2C197E52C
:10711000B64668845EB510999CBD560F41ED16E8E1
:107120007561891C76049BBB6E651A9CB2A7FE84B0
:1071300035095F1B890FF76C35B13DB00EB6055EA2
:1071400004928C9866329D7EF4F8EDDF5B981C37D4
:1071500076ACCEAD7E4C6482F8283574E207D2BDA1
:107160006067196CA7C1538FF9AF877056634437B6
:107170004FF7694B4E44494058D01561BEEFD5F4E6
:10718000E01D255197460D15237925EA5BDF746FC5
:107190009522645C7F32EFF59E7B4B0ADC6D58D5FF
:1071A0007347BD5A93DE7F8808FB47B8E8763E1FD9
:1071B000F1DA1CF9CAA2529BE2F19D41F9710A571A
:1071C0001B0A2A8CD2E1FB91B8B0770D01D038614F
:1071D000681FEA23638C3D0C46294AF711E22B44D1
:1071E0006EC4CF0E179C6DFC47EA9AF09B90E24963
:1071F0009A20210106AD4FEA06FC52C27B7AEEF5D9
:107200006DC03A858297D88B8F00FF92A1DD4745EC
:107210002DF5AEE7D18933B50C967FF15F1A024C9C
:107220007AEDFAC6664A4EFD8918808AB01A513C3A
:107230001D14BE57BDE2BA161A0184C448EC28CF0B
:107240006E03950345BB5F1D1E7D64F40A143E82E8
:107250006E9EE02A0B7ACAA534F878E36F0F694E68
:10726000597EFA824000BC2F477773B3DDBAFCA980
:10727000A9D5477C0CBB28494358916F77FA7E38D3
:107280006E5A1B7B9B0ED3EE56C68B912D4FCC4571
:1072900046750C2714D34FFFBA47715A2D3071E051
:1072A000EFD846018FF5C25758BA8B53231E506F43
:1072B00044FFCE76741D3473BBEAD36287F75BBBA1
:1072C000934426BDF45B516DA046F25F0B05EFC6FB
:1072D000F4344EEACAC298EEBCF3F76F2B9D782DBA
:1072E00046F98949BD7C45E67BEFEAD555A92232AE
:1072F000D618D3603A90AF3DE84ABECE3C5FCA5440
:107300003C38C77414EC67FA56174AD1FE51E5D3DE
:10731000AEE64CEF48B03B51D981850C32C584F1C3
:10732000EA191301944282CC01B35662BB0DDB1AF9
:107330001B9C73615C978F3F3C1ACC1FA624EA907C
:10734000064AD6FE14734436AA475886A627024A30
:107350005317E391629E681BBD238550D54E84224E
:107360004D51D1E42C70292AB2327225DBF3C6705C
:10737000BEE077C65F3CCD09732B02B82F51BB210D
:107380008C73AB8B01D9E5DDB788BF15231E0F4881
:107390004C14DDCBE06F0A94D381C0EC07BBB95429
:1073A00060348FCA35486984383070E8FEB5F14BD7
:1073B000309DFCD07BA3B16BD709689D87F1E1D2EA
:1073C000808A59EB3B5EB9BC685CF5592B918165AD
:1073D00075E7E75ECC52824B9E1B1214DD4ACB98B8
:1073E000A811349228AF76F1BA9C098F1B7C40F922
:1073F00050061A045F8B628989427456147D75EEBB
:107400007BD1904577E761053534E4B02878753253
:1074100098A2AEA6B4C776C0CBB6A35E9087250E61
:107420006A3B72CABC1CC075236136FD5B152FA771
:10743000F518631E958B8F8F434D5E33A119A453AE
:10744000B8A2FAE3885FD761EF05A5788AA0216F1B
:1074500020DAE3245A79A7520C78306369D6518434
:10746000D73770B738B6CC5798CF241189FDD5E9F6
:10747000B7DE2F494C85042BD350593361B795A300
:10748000809F0F0D003B0F1561894F9C7AC2685D8C
:10749000A6585813D2ADADED354857410C466B1286
:1074A0000B7313443E7F773066C10679D1A668E23C
:1074B00039756B52DBE3F94E881486D39783210F1D
:1074C000824F59D76AD390797100295DB838984DA9
:1074D000B33DA6CFC6E35B9C1FF9D400C6889C06CB
:1074E0002795FE15D70B288D2585FE1D48893AFF67
:1074F00009F43693CD5E58F43BBEFA0424B5A44C8F
:10750000062CE884667E51CAC4A2C2F276E16034D9
:1075100014E1A92DC631682635BFE02C5476A4DAD3
:10752000FF9969F7E03188A8D4B61759CC90995ED5
:10753000E8439D86A8A79C79E3E233EDCF85684FA9
:10754000A9CAEA720F61F008E9A7C847B3DCFB8A51
:10755000E6EF1972F0016BF7DB87B36928F6942C1C
:107560000D2F2B7522860B860953469D510315322C
:107570000B1A1DE6200243E2FC0A0E06385050208A
:1075800080ABB712D46C70B53D4BD772B37104CDDC
:10759000CD68666E3D974A2865253F87B64ACBB6CB
:1075A00078214318281DC65627538E8CD12673D5B3
:1075B000777E50C7A9C7BD0B9254102D6177B7E0F5
:1075C0003D078CF2174885700D14A3FBA2B5022964
:1075D0002725D000F3D2FE29BFF22224A2A4B8AE00
:1075E00064EE0330C998BC31BB93ED5BA2C80EDAE0
:1075F000490EC70A2CC0B7AB3FB14159AF0E1A3D77
:107600008B6864EAD5E91735822B3A3A2B59203A30
:1076100003A89953CE6BE5766BC573C5DFF668AAF0
:10762000C6C112F2B5A833A38F49A6A28B111E546E
:10763000AC300DF70FA7181E5C105A9DBA62D2AF7E
:107640009B1A782A3D64F9E99BF87D6CE37E2477E8
:10765000DE9E3CF7467C4131EEAAA2109263A36BFA
:10766000219FBC7A0D8A2F6708240A344B5255FBA0
:10767000377C8849D3FD9603C74C14D8EEA37ED53A
:10768000E810AB20149147997A2B7E8085FF7075A6
:107690008B5919CBC2BC136B7C384E4A58D8956EA7
:1076A000FE474F1C707A07A3C79EFDA4FE2EAFEACB
:1076B000A257AD1ACE6BB485F3C208FDCC7261D966
:1076C000A1F5CF2152AF7A2C914897C68754C2AF0B
:1076D00000289509AE278A0C04550F826A82179BF1
:1076E000AF7F8A0C6A3DF9130AE1FF04FAC333C184
:1076F000D422A9AFC2112B72CECAE7A6D66B6653AD
:10770000DE5AF2E3E4DEB5FAB19247BF42A4702537
:10771000ECFB0247A294C599E57A73096994A06DC0
:10772000846E9999692BCA324432271CDC3A633A39
:10773000092A9120F130E03244226FFC22C8FF8DEB
:10774000E213E1AB67CF041A9B473F2AAE4CFF8799
:10775000A8703454A9BE58BAF81AB302D839B00E7A
:1077600084B5E31B30B6AD23207DD5DC4B35C85D39
:10777000DC915E31617C69327D529D39DABCD2E99F
:10778000FE057209B35BF9FEA4CA4685FC35D8D262
:10779000C4D4A65CC9E7B4E5012A605D72B482F581
:1077A00073712038CA7EF59430DC1F8B9F2527A487
:1077B000243AE08BDADED6C105E256E99A27A288A0
:1077C0003285D230C8E2BC580004A99D8F325C9942
:1077D00041BD0D193CF487D2ECBD274AACD983BA20
:1077E0001242FB420773ED5B16457BF4D81312DFA0
:1077F000F1E5787B25993842EDB578857E37B195EE
:10780000C2E73F61633FB5F4636AADA2795DD8B664
:10781000D9BA823F0C12ADF9EE7F35AB58A5CA9E9E
:1078200078FCC761C158E42B431181F68E764BD3A7
:10783000C079E08C49E6E37F27D61BF576FA89AC60
:107840004E9824BAD63220F1434F4E5F5A13BC3BB8
:10785000ADD5A1F3587369BF653D00CC2D38A0C4E8
:10786000014F1DD8B6852B3C5D08D8F75A59EAF36D
:10787000605012D9029D6F6928B0B3D89C7700166A
:1078800017E33697D35F5D87BAC1B7721FF4FA7FEB
:10789000F1876E5C208AF1E9FCA602763CD71A7368
:1078A000FEFA75532219BF699DB3192992318D11C2
:1078B000B240C80115C186F6D3783D64E5272DDFB7
:1078C0001FA6E26AA3F267D4B0EBA390EB24DBCB54
:1078D0004ECB55994F7A9E6157FD126BBAE02B0E35
:1078E000F8B2B7951A0F3D14315AF5E3096A675A91
:1078F000E58A690BFC97A1FD1DB256C671FE2731C2
:10790000175531DA04A9ABC36D0661A6035C7DB6D9
:107910007EE9EC999A73643CDA7EA0FEECB3351FE5
:10792000221C731BF8E55ECD55A8E4522F7383B675
:107930006BB47F008E44C2752659BD49DEF78D6E4B
:107940005E8081FF63A61830144CBCA5C95BE4B20D
:1079500077649C85CD7A51C03FF4BCA03F93578695
:10796000EFC62248FF201CE5004FE6DBB7BECFB8CC
:107970008C99914DC75A9FB5547731241C80A088AB
:10798000D7C1CAB4605042340117FF546423E15494
:10799000F797EFD0121E4A0943E65389B9C212D1B4
:1079A00024C6D872A1BFB152A75E92FDE0548A529C
:1079B0003D1587EB98B03A15046F160A51CFE57A5A
:1079C0009F2DA75C536FA96FDB1C59BCE8897DD242
:1079D00069F7274B1EAB918A3C3BEDD5B183F5BDD2
:1079E00097E2C57EA11210C6A924A889E9B655E17F
:1079F000452CADA74A9A933E9F4CA6B1289CC4CD76
:107A0000A6D5CA7E2C9E29F9E1CEE3C56B04049568
:107A100032CD66203CBFAF826D46A627F50B3C46B3
:107A2000C643DA3FD059FABE16A7E996482ABB8961
:107A3000468689DFAFB2892BB4236A78E0474A755E
:107A40000D553AFA00BCDF5450A957470D58D8409D
:107A5000FE85044FE77D51B4C478ECFFDC1392A39C
:107A6000FEE39EBEACA449E4D0EA722324E57BD1B8
:107A70005F1817A4CD55A36F213D7D8633B0115AF1
:107A80005212A722DE11A84A305BF96C2811EA6174
:107A9000132264DFA15F11D1041733E46713A650EA
:107AA0000111236FD59A93CB3A06AFECAF69F7D7A4
:107AB0006A78ECC081BAF2A2A517C0E7A8E7EE4E3B
:107AC000FEFE9FCB8D470932177DA62D399E473D7F
:107AD000267AD8A73E31518E91169C50DD6365AC55
:107AE000C0A6BD6B3EEDB01EDB52BB8E8E0379107F
:107AF0005118EBCE4DB59681469BE7725833711401
:107B00006D8A5E508FB7AEDF926605F4E0D948CB40
:107B1000E68E4E3E4E714C64B726DA09D3881FCAF2
:107B2000057D1536AEC34936DB6A21F37A9A11E238
:107B300043A491AEAFE5FC9C7F6D52753F72CED3EE
:107B4000D23DD278A4761E1B1DEA99A35AA980A023
:107B50007825D9D6D9A52ECE8BFFF0AE25983DC37A
:107B60002BF5EC0F4F39BB80C85341EA0C415D1E29
:107B70009FE484D8F44BF4992C2C44DE24BEB6F058
:107B80001370679D7078C704CEF0AFC9C17FBB3C4E
:107B9000486C2A06BC4C9CEAE2FBDEB89BBF2BCAB1
:107BA00051F2A5A118EF3B9C365FC5E080E234940A
:107BB000C42FCBC9BA19438EB7552659DEA0FE3E55
:107BC000F987E0058C446413A595F58E1CAF9DAC38
:107BD000EAEE88CB982C6FC074272DD4850A7B17CA
:107BE0001B20549BA3E79BA703BA6D0B4B67C69062
:107BF00062E8A610DF6960A22EEAB42F0CF28E7044
:107C000008E14922194BF4F8456B359502567D720F
:107C1000F7EE03A622E4A61237943838E1C7A48A07
:107C2000C05FF66075F3CFB1C5CCAF18D51F9D16F8
:107C30006DB30BEADD2368A85F0A5C82920BF51531
:107C40008CEED1A08DCEB5E31BD5EEF8B39776B808
:107C5000ACB750EA22FE25B9DC1125CB226C368167
:107C6000ED01F1F25FCA528604F324609359FB518F
:107C700065E4EE57C76FFAF12579941CA909946A57
:107C8000DD42E8FB5658783501F62321B08AB6DF8D
:107C9000FA8B15A31F6519148EC59797991C7B70D5
:107CA00025498BA6266789C03CFC782896765F66B6
:107CB0003ACA0550F8D42A7897D2BF92F858A5133B
:107CC0006DF98025B2B15FB84E28A3D19494110C00
:107CD00040CA6402D633AF4C3E6913A4AB7623F599
:107CE000C0640B829D4FAA03ED47CCEC16E2B9BFEE
:107CF000F7D353F25717E050842856C1807DEE69C0
:107D00003BCEC3B01E2F1EB547B2E9497F2938D2FA
:107D1000B316A96EC7C4EDD10E83716803549E3F9C
:107D2000A7D8580A10E2940BE4C924865B7A270A84
:107D30000A801518689E05AE10986F3BCA80987D22
:107D4000B3FA20E3B15CC08A0C65E9F957FED25D55
:107D5000CFB077D08A2066A9172930189CC1C059A6
:107D60005849E7BE939291678555A11B3CCA1A7288
:107D7000A25D2EF60304050A08060BFF0209070D93
:107D8000010C00FF2025692025692025692D256922
:107D900000202025633A256900202020205F5F7C99
:107DA000002C00610044697370206F66660D0A0044
:107DB000555345520046004700424547494E005240
:107DC000414400442E4D590043005052474D005548
:107DD00053455220202000662020006720200042CA
:107DE0004547494E20202020200052414420202099
:107DF00000442E4D592020200043202020000D0C4F
:107E0000205A2F3C00000500000003072061693B59
:107E10000000FFFFFFFF4D000000C4400000000015
:107E2000000081100000DC400000E1400000DF4065
:107E30000000FF00000059080000EB400000F54082
:107E40000000934000000000000079060000074198
:107E50000000E1400000134100000000000019078D
:107E6000000015410000E140000021410000000039
:107E70000000B108000023410000E140000044413F
:107E80000000000000004106000046410000E14003
:107E900000000F000000F4010000040103010201D2
:107EA000010411040F041704160118010000CF7D0E
:107EB0000000D77D0000DB7D0000DF7D0000B77D86
:107EC0000000EA7D0000F17D0000F97D0000CA7D20
:107ED0000000081C242C4448586C74050205080452
:107EE000080B08040405010504090809040608072D
:107EF0000206020402060106040701030803040C3B
:107F0000080D020C0203020C010C040D010D080DFA
:107F10000408020808070802020704080108040907
:107F20000209010A080B020A0201080A010A040BED
:107F300001020802041008110210021108100110B9
:107F4000041101120212011302130812080F081281
:107F50000413011304140214011502150814081760
:107F6000081404150115041702170119081A02193B
:107F7000021602190119041A01160816041B021B25
:107F8000081A0818021A041B011B04180818040B0D
:107F9000042020202020202020202000000001009C
:107FA0000000B07D0000B57D0000B77D0000B97D08
:107FB0000000B77D0000BF7D0000C37D0000C87DCC
:067FC0000000CA7D000074
:00000001FF
